:0407000055EF54F06D
:08070800046ED8CF05F0E0CF2C
:1007100006F00001E9CF0CF0EACF07F0E1CF08F0D6
:10072000E2CF09F0D9CF0AF0DACF0BF0F3CF12F015
:10073000F4CF13F0FACF14F0FBCF15F000C00EF099
:1007400001C00FF002C010F003C011F0A3AAACEF7B
:1007500003F0A4BA53EF0FF09DAAB2EF03F09EBAD4
:1007600009EF0FF00EC000F00FC001F010C002F052
:1007700011C003F00CC0E9FF07C0EAFF078E08C0F4
:10078000E1FF09C0E2FF0AC0D9FF0BC0DAFF12C0C7
:10079000F3FF13C0F4FF14C0FAFF15C0FBFF0450B1
:1007A00006C0E0FF05C0D8FF1000F2CF0DF0F29EAA
:1007B000F76AC80FF66E070EF722000EF86E0900F2
:1007C000F5500DBEF28E1200280C0106F2CF0DF08E
:1007D000F29EF76AEA0FF66E070EF722000EF86E29
:1007E0000900F5500DBEF28E1200446961676E6F0C
:1007F00073746963204D6F64653A204F6E00F2CFC9
:100800000DF0F29EF76A1C0FF66E080EF722000E2E
:10081000F86E0900F5500DBEF28E12004469616752
:100820006E6F73746963204D6F64653A204F66661E
:100830000000F2CF0DF0F29EF76A500FF66E080E30
:10084000F722000EF86E0900F5500DBEF28E120070
:10085000486F73742053657269616C20496E7075BE
:10086000743A20456E61626C65640000F2CF0DF051
:10087000F29EF76A8A0FF66E080EF722000EF86EE7
:100880000900F5500DBEF28E1200486F73742053AC
:10089000657269616C20496E7075743A20446973A1
:1008A00061626C656400F2CF0DF0F29EF76AC40FCE
:1008B000F66E080EF722000EF86E0900F5500DBE18
:1008C000F28E120053657269616C204563686F3A5D
:1008D00020456E61626C65640000F2CF0DF0F29EFF
:1008E000F76AF80FF66E080EF722000EF86E090090
:1008F000F5500DBEF28E120053657269616C204591
:1009000063686F3A2044697361626C656400F2CF7A
:100910000DF0F29EF76A2C0FF66E090EF722000E0C
:10092000F86E0900F5500DBEF28E120047656E6C30
:100930006F636B204D6F64653A20456E61626C6534
:100940006400F2CF0DF0F29EF76A600FF66E090EAA
:10095000F722000EF86E0900F5500DBEF28E12005F
:1009600047656E6C6F636B204D6F64653A20446918
:100970007361626C65640000F2CF0DF0F29EF76A5D
:10098000960FF66E090EF722000EF86E0900F5506C
:100990000DBEF28E12000000F2CF0DF0F29EF76A4B
:1009A000B60FF66E090EF722000EF86E0900F5502C
:1009B0000DBEF28E1200465047412054756E6E6592
:1009C0006C3A2041637469766500F2CF0DF0F29EB7
:1009D000F76AE80FF66E090EF722000EF86E0900AE
:1009E000F5500DBEF28E1200465047412054756EF0
:1009F0006E656C3A20496E61637469766500F2CF6A
:100A00000DF0F29EF76A1C0FF66E0A0EF722000E2A
:100A1000F86E0900F5500DBEF28E12004E6F20499F
:100A20006E70757420202020202020200000F2CF3E
:100A30000DF0F29EF76A4C0FF66E0A0EF722000ECA
:100A4000F86E0900F5500DBEF28E120048442031B8
:100A500030383070203630487A2020200000F2CF25
:100A60000DF0F29EF76A7C0FF66E0A0EF722000E6A
:100A7000F86E0900F5500DBEF28E12004844203188
:100A800030383070203530487A2020200000F2CFF6
:100A90000DF0F29EF76AAC0FF66E0A0EF722000E0A
:100AA000F86E0900F5500DBEF28E12004844203158
:100AB000303830692035392E3934487A0000F2CF89
:100AC0000DF0F29EF76ADC0FF66E0A0EF722000EAA
:100AD000F86E0900F5500DBEF28E12004844203128
:100AE00030383069203530487A2020200000F2CF9D
:100AF0000DF0F29EF76A0C0FF66E0B0EF722000E49
:100B0000F86E0900F5500DBEF28E12004844202008
:100B100037323050202035392E3934487A00F2CF20
:100B20000DF0F29EF76A3C0FF66E0B0EF722000EE8
:100B3000F86E0900F5500DBEF28E120048442020D8
:100B40003732305020203530487A20202000F2CF34
:100B50000DF0F29EF76A6C0FF66E0B0EF722000E88
:100B6000F86E0900F5500DBEF28E12004856203185
:100B70003630307831323030203630487A00F2CF9B
:100B80000DF0F29EF76A9C0FF66E0B0EF722000E28
:100B9000F86E0900F5500DBEF28E12004856203155
:100BA0003430307831303530203630487A00F2CF6A
:100BB0000DF0F29EF76ACC0FF66E0B0EF722000EC8
:100BC000F86E0900F5500DBEF28E12004856203125
:100BD0003336367820373638203630487A00F2CF30
:100BE0000DF0F29EF76AFC0FF66E0B0EF722000E68
:100BF000F86E0900F5500DBEF28E120048562031F5
:100C00003238307820373638203630487A00F2CF04
:100C10000DF0F29EF76A2C0FF66E0C0EF722000E06
:100C2000F86E0900F5500DBEF28E120048562031C4
:100C30003032347820373638203630487A00F2CFD8
:100C40000DF0F29EF76A5C0FF66E0C0EF722000EA6
:100C5000F86E0900F5500DBEF28E120048562020A5
:100C60003830307820363030203630487A00F2CFB5
:100C70000DF0F29EF76A8C0FF66E0C0EF722000E46
:100C8000F86E0900F5500DBEF28E12004856202075
:100C90003634307820343830203735487A00F2CF77
:100CA0000DF0F29EF76ABC0FF66E0C0EF722000EE6
:100CB000F86E0900F5500DBEF28E1200534420204C
:100CC000343830692032392E3937487A0000F2CF73
:100CD0000DF0F29EF76AEC0FF66E0C0EF722000E86
:100CE000F86E0900F5500DBEF28E1200534420201C
:100CF00035373669203235487A2020200000F2CF7F
:100D00000DF0F29EF76A1C0FF66E0D0EF722000E24
:100D1000F86E0900F5500DBEF28E12002000F2CFE1
:100D20000DF0F29EF76A3C0FF66E0D0EF722000EE4
:100D3000F86E0900F5500DBEF28E120048562031B3
:100D40003932307831323030203630487A00F2CFC4
:100D50000DF0F29EF76A6C0FF66E0D0EF722000E84
:100D6000F86E0900F5500DBEF28E12004856203183
:100D70003238307831303234203630487A00F2CF91
:100D80000DF0F29EF76A9C0FF66E0D0EF722000E24
:100D9000F86E0900F5500DBEF28E12004856202064
:100DA0003634307820343830203630487A00F2CF6C
:100DB0000DF0F29EF76ACC0FF66E0D0EF722000EC4
:100DC000F86E0900F5500DBEF28E1200204D6173D1
:100DD00074657220506F776572204F666600F2CF9F
:100DE0000DF0F29EF76AFC0FF66E0D0EF722000E64
:100DF000F86E0900F5500DBEF28E1200204D6173A1
:100E000074657220506F776572204F6E0000F2CFCC
:100E10000DF0F29EF76A2C0FF66E0E0EF722000E02
:100E2000F86E0900F5500DBEF28E12002020496EBA
:100E30007075743120287950625072290000F2CF09
:100E40000DF0F29EF76A5C0FF66E0E0EF722000EA2
:100E5000F86E0900F5500DBEF28E12002020496E8A
:100E600070757432202848442D5344492900F2CF2C
:100E70000DF0F29EF76A8C0FF66E0E0EF722000E42
:100E8000F86E0900F5500DBEF28E120020204F754D
:100E90007470757431202879506250722900F2CF35
:100EA0000DF0F29EF76ABC0FF66E0E0EF722000EE2
:100EB000F86E0900F5500DBEF28E120020204F751D
:100EC00074707574322848442D5344492900F2CF78
:100ED0000DF0F29EF76AEC0FF66E0E0EF722000E82
:100EE000F86E0900F5500DBEF28E120020436C65BD
:100EF0006172696E6720416C6C2020200000F2CF87
:100F00000DF0F29EF76A1C0FF66E0F0EF722000E20
:100F1000F86E0900F5500DBEF28E12002052657376
:100F2000746172742053797374656D200000F2CF80
:100F30000DF0F29EF76A4C0FF66E0F0EF722000EC0
:100F4000F86E0900F5500DBEF28E12002020536895
:100F50007574646F776E2041637469766520000054
:100F6000F2CF0DF0F29EF76A7E0FF66E0F0EF722AB
:100F7000000EF86E0900F5500DBEF28E1200202012
:100F80002053595354454D204D454E5520200000C7
:100F9000F2CF0DF0F29EF76AAE0FF66E0F0EF7224B
:100FA000000EF86E0900F5500DBEF28E12002020E2
:100FB0002053657269616C20496E70757420000061
:100FC000F2CF0DF0F29EF76ADE0FF66E0F0EF722EB
:100FD000000EF86E0900F5500DBEF28E12002020B2
:100FE0002053657269616C204563686F20200000A2
:100FF000F2CF0DF0F29EF76A0E0FF66E100EF7228A
:10100000000EF86E0900F5500DBEF28E1200202081
:1010100020436C656172204D656D6F727920000010
:10102000F2CF0DF0F29EF76A3E0FF66E100EF72229
:10103000000EF86E0900F5500DBEF28E1200202051
:101040002047656E4C6F636B204D6F646520000018
:10105000F2CF0DF0F29EF76A6E0FF66E100EF722C9
:10106000000EF86E0900F5500DBEF28E1200202021
:1010700020465047412054756E6E656C202000005C
:10108000F2CF0DF0F29EF76A9E0FF66E100EF72269
:10109000000EF86E0900F5500DBEF28E12002020F1
:1010A00020494E5055542031204D454E55200000CA
:1010B000F2CF0DF0F29EF76ACE0FF66E100EF72209
:1010C000000EF86E0900F5500DBEF28E12002020C1
:1010D00048442F48562F5344202020496E200000BA
:1010E000F2CF0DF0F29EF76AFE0FF66E100EF722A9
:1010F000000EF86E0900F5500DBEF28E1200202091
:1011000048442F48562F53442020204F7574000028
:10111000F2CF0DF0F29EF76A2E0FF66E110EF72247
:10112000000EF86E0900F5500DBEF28E1200202060
:1011300048442D5344492F534449204F75740000AF
:10114000F2CF0DF0F29EF76A5E0FF66E110EF722E7
:10115000000EF86E0900F5500DBEF28E1200202030
:1011600020494E5055542032204D454E5520000008
:10117000F2CF0DF0F29EF76A8E0FF66E110EF72287
:10118000000EF86E0900F5500DBEF28E1200202000
:1011900048442D5344492F53444920496E200000B0
:1011A000F2CF0DF0F29EF76ABE0FF66E110EF72227
:1011B000000EF86E0900F5500DBEF28E12002020D0
:1011C0005247424856204F5554204D454E55000039
:1011D000F2CF0DF0F29EF76AEE0FF66E110EF722C7
:1011E000000EF86E0900F5500DBEF28E12002020A0
:1011F000486F72697A6F6E74616C20202020000045
:10120000F2CF0DF0F29EF76A1E0FF66E120EF72265
:10121000000EF86E0900F5500DBEF28E120020206F
:10122000566572746963616C2020202020200000C4
:10123000F2CF0DF0F29EF76A4E0FF66E120EF72205
:10124000000EF86E0900F5500DBEF28E120020203F
:101250004F7574206E6F742052474248562000002C
:10126000F2CF0DF0F29EF76A7E0FF66E120EF722A5
:10127000000EF86E0900F5500DBEF28E120020200F
:101280002020496E7075742031204D656E75000008
:10129000F2CF0DF0F29EF76AAE0FF66E120EF72245
:1012A000000EF86E0900F5500DBEF28E12002020DF
:1012B0002020496E7075742032204D656E750000D7
:1012C000F2CF0DF0F29EF76ADE0FF66E120EF722E5
:1012D000000EF86E0900F5500DBEF28E12002020AF
:1012E00020205247424856204F757420506F73009B
:1012F000F2CF0DF0F29EF76A0E0FF66E130EF72284
:10130000000EF86E0900F5500DBEF28E120020207E
:10131000202053797374656D204D656E7520000033
:10132000F2CF0DF0F29EF76A3E0FF66E130EF72223
:10133000000EF86E0900F5500DBEF28E120020204E
:1013400020205374616E646279204D6F64650000E3
:10135000F2CF0DF0F29EF76A6E0FF66E130EF722C3
:10136000000EF86E0900F5500DBEF28E120020201E
:1013700020202020537461727400F2CF0DF0F29E91
:10138000F76A980FF66E130EF722000EF86E09003A
:10139000F5500DBEF28E1200202020202020205972
:1013A00065730000F2CF0DF0F29EF76AC20FF66E81
:1013B000130EF722000EF86E0900F5500DBEF28EE6
:1013C000120020202020202020204E6F0000F2CF8D
:1013D0000DF0F29EF76AEC0FF66E130EF722000E78
:1013E000F86E0900F5500DBEF28E1200202020206C
:1013F000202020204F6E0000F2CF0DF0F29EF76A01
:10140000160FF66E140EF722000EF86E0900F55056
:101410000DBEF28E1200202020202020204F666674
:101420000000F2CF0DF0F29EF76A400FF66E140E38
:10143000F722000EF86E0900F5500DBEF28E120074
:10144000202046617374204F6E00F2CF0DF0F29EA3
:10145000F76A680FF66E140EF722000EF86E090098
:10146000F5500DBEF28E12002020536C6F77204F86
:101470006E00F2CF0DF0F29EF76A900FF66E140E2A
:10148000F722000EF86E0900F5500DBEF28E120024
:1014900020204E6F20496E7075742020202020205F
:1014A0000000F2CF0DF0F29EF76AC00FF66E140E38
:1014B000F722000EF86E0900F5500DBEF28E1200F4
:1014C0002020484420313038307020363020202011
:1014D0000000F2CF0DF0F29EF76AF00FF66E140ED8
:1014E000F722000EF86E0900F5500DBEF28E1200C4
:1014F00020204844203130383070203530202020E2
:101500000000F2CF0DF0F29EF76A200FF66E150E76
:10151000F722000EF86E0900F5500DBEF28E120093
:10152000202048442031303830692035392E393474
:101530000000F2CF0DF0F29EF76A500FF66E150E16
:10154000F722000EF86E0900F5500DBEF28E120063
:101550002020484420313038306920353020202088
:101560000000F2CF0DF0F29EF76A800FF66E150EB6
:10157000F722000EF86E0900F5500DBEF28E120033
:10158000202048442020373230702035392E39341D
:101590000000F2CF0DF0F29EF76AB00FF66E150E56
:1015A000F722000EF86E0900F5500DBEF28E120003
:1015B0002020484420203732307020353020202031
:1015C0000000F2CF0DF0F29EF76AE00FF66E150EF6
:1015D000F722000EF86E0900F5500DBEF28E1200D3
:1015E0002020485631363030783132303020363095
:1015F0000000F2CF0DF0F29EF76A100FF66E160E95
:10160000F722000EF86E0900F5500DBEF28E1200A2
:101610002020485631343030783130353020363063
:101620000000F2CF0DF0F29EF76A400FF66E160E34
:10163000F722000EF86E0900F5500DBEF28E120072
:101640002020485631333636782037363820363029
:101650000000F2CF0DF0F29EF76A700FF66E160ED4
:10166000F722000EF86E0900F5500DBEF28E120042
:1016700020204856313336307820373638203630FF
:101680000000F2CF0DF0F29EF76AA00FF66E160E74
:10169000F722000EF86E0900F5500DBEF28E120012
:1016A00020204856313238307831303234203630CC
:1016B0000000F2CF0DF0F29EF76AD00FF66E160E14
:1016C000F722000EF86E0900F5500DBEF28E1200E2
:1016D00020204856313238307820383030203630AB
:1016E0000000F2CF0DF0F29EF76A000FF66E170EB3
:1016F000F722000EF86E0900F5500DBEF28E1200B2
:10170000202048563132383078203736382036306D
:101710000000F2CF0DF0F29EF76A300FF66E170E52
:10172000F722000EF86E0900F5500DBEF28E120081
:101730002020485631303234782037363820363041
:101740000000F2CF0DF0F29EF76A600FF66E170EF2
:10175000F722000EF86E0900F5500DBEF28E120051
:10176000202048562038303078203630302036302F
:101770000000F2CF0DF0F29EF76A900FF66E170E92
:10178000F722000EF86E0900F5500DBEF28E120021
:1017900020204856203634307820343830203630F7
:1017A0000000F2CF0DF0F29EF76AC00FF66E170E32
:1017B000F722000EF86E0900F5500DBEF28E1200F1
:1017C00020204E54534320532D566964656F2020CA
:1017D0000000F2CF0DF0F29EF76AF00FF66E170ED2
:1017E000F722000EF86E0900F5500DBEF28E1200C1
:1017F000202050414C20532D566964656F202020D5
:101800000000F2CF0DF0F29EF76A200FF66E180E70
:10181000F722000EF86E0900F5500DBEF28E120090
:1018200020204E54534320436F6D706F736974656D
:101830000000F2CF0DF0F29EF76A500FF66E180E10
:10184000F722000EF86E0900F5500DBEF28E120060
:10185000202050414C20436F6D706F736974652078
:101860000000F2CF0DF0F29EF76A800FF66E180EB0
:10187000F722000EF86E0900F5500DBEF28E120030
:1018800020204E6F204F757470757420202020200A
:101890000000F2CF0DF0F29EF76AB00FF66E180E50
:1018A000F722000EF86E0900F5500DBEF28E120000
:1018B00020204856313932307831323030203630BD
:1018C0000000F2CF0DF0F29EF76AE00FF66E180EF0
:1018D000F722000EF86E0900F5500DBEF28E1200D0
:1018E00020205344204E54534320202020202020E9
:1018F0000000F2CF0DF0F29EF76A100FF66E190E8F
:10190000F722000EF86E0900F5500DBEF28E12009F
:10191000202053442050414C202020202020200013
:10192000F2CF0DF0F29EF76A3E0FF66E190EF72217
:10193000000EF86E0900F5500DBEF28E1200202048
:1019400048442031303830702033302020200000CF
:10195000F2CF0DF0F29EF76A6E0FF66E190EF722B7
:10196000000EF86E0900F5500DBEF28E1200202018
:10197000484420313038307020323520202000009B
:10198000F2CF0DF0F29EF76A9E0FF66E190EF72257
:10199000000EF86E0900F5500DBEF28E12002020E8
:1019A00053442020343830692032392E3937000032
:1019B000F2CF0DF0F29EF76ACE0FF66E190EF722F7
:1019C000000EF86E0900F5500DBEF28E12002020B8
:1019D000534420203537366920323520202000003E
:1019E0000A0D55315F4953522030302030302030BD
:1019F000302025325820253258000A0D55315F49D4
:101A000053522D455252203030203030203030207B
:101A1000253258205B2532585D000A0D55315F494B
:101A200053522D455252203030203030203030205B
:101A3000253258205B2532585D000A0D55315F492B
:101A400053522D455252203030203030203030203B
:101A50005B2532585D20253258000A0D55315F490B
:101A600053522D455252203030203030203030201B
:101A70005B2532585D20253258000A0D50726F6484
:101A8000756374204E616D653A20257325730A0DC8
:101A9000000020202020436F6D70696C65643A203F
:101AA00025732061742025730A0D000030392D4AFA
:101AB000756E2D31300031373A33323A323700000B
:101AC000496E70757420313A2025732C00004F75D3
:101AD0007470757420313A2025732C004F75747022
:101AE000757420323A2025730A0D0000496E707516
:101AF0007420323A2025732C00004F757470757471
:101B000020313A2025732C004F7574707574203283
:101B10003A2025730A0D00000A0D436F6D6D616E4A
:101B20006420436F6D706C6574650A0D3E000A0D8C
:101B3000436F6D6D616E6420436F6D706C6574658D
:101B40000A0D3E000A0D436F6D6D616E6420436F98
:101B50006D706C6574650A0D3E003E2573204E6FF6
:101B60007420466F756E640A0D3E00000A0D436FC7
:101B70006D6D616E6420436F6D706C6574650A0DE8
:101B80003E000A0D44696167203D204F6E0A0D003A
:101B90000A0D44696167203D204F66660A0D00000A
:101BA0000A0D506F776572203D204F6E0A0D0000C0
:101BB0000A0D506F776572203D204F66660A0D0052
:101BC0000A0D496E707574203D20496E7075742041
:101BD000310A0D000A0D496E707574203D20496E62
:101BE00070757420320A0D000A0D496E70757420EC
:101BF0003D204E2F410A0D000A0D4F75747075740B
:101C0000203D20310A0D00000A0D4F757470757467
:101C1000203D20320A0D00000A0D46504741205455
:101C2000756E6E656C204163746976650A0D0000FF
:101C30000A0D465047412054756E6E656C20416315
:101C4000746976650A0D00000A0D53657269616C4E
:101C50004563686F203D205965730A0D00000A0D29
:101C600053657269616C4563686F203D204E6F0A51
:101C70000D002042746E282532782F2575292D47B6
:101C8000727031200A0D00002D47727034285461A3
:101C9000736B293A2042746E282532782F257529D6
:101CA0000A0D0000555848442043726F7373706FDB
:101CB000696E7425730A0D0020202020436F6D701B
:101CC000696C65643A2025732061742025730A0DC0
:101CD000000030392D4A756E2D31300031373A33DE
:101CE000323A323700000A0D436F6D6D616E642029
:101CF000436F6D706C6574650A0D3E000A0D4650A9
:101D000047412D5243563A2000000D0A576169742D
:101D1000465047415F526573706F6E736528292086
:101D200054696D656F757420254C7520286D732975
:101D300000000D0A57616974465047415F52657350
:101D4000706F6E7365282920446174612052656349
:101D5000656976656420254C7520286D732900001F
:101D60000A0D465047412D534E443A2025327820E3
:101D700025327820253278202532782025327820A7
:101D80002532782025327820253278202532782097
:101D90002532780A0D000A0D465047412D534E4416
:101DA0003A202532782025327820253278202532B5
:101DB0007820253278202532782025327820253267
:101DC0007820253278202532780A0D000A0D5472C9
:101DD0006163652825642920465047412D534E44B0
:101DE0003A20253278202532782025327820253275
:101DF000782025327820253278202532780A0D0087
:101E0000A4A8FED76D6E14EF0FF09EA8FED7AD6E9E
:101E1000000C0801066B1EA00AD09EAAFED7AECF0A
:101E200006F806510001ECD73BD03AD008019EAA33
:101E3000FED7AECF06F80651080803E006517F082A
:101E400009E1080E0001E1DF200EDFDF080EDDDF13
:101E500027D00801036A0001DB518A0FE96E000EEA
:101E60000320EA6E06C8EFFFDCC005F8010EDB2593
:101E7000500802E2DB6B01D0DB2BDB51DC5D02E1C1
:101E800005C8DBF0080106510D0803E10001892BAC
:101E900008014DA403D006510001B7DF0001DD8128
:101EA0009E9AB2EF03F00801066B1EA00AD0A4AA06
:101EB000FED76ECF06F806510001A7DF25D024D04B
:101EC0000801A4AAFED76ECF06F8036A01011E51CD
:101ED000DE0FE96E000E0320EA6E06C8EFFF1FC199
:101EE00005F8010E1E253F0802E21E6B01D01E2BD5
:101EF0001E511F5D02E105C81EF10801063D02D01A
:101F00000101202B0001DD83A49AB2EF03F006014A
:101F1000106703D0116702D007D0112B0FC6EEFF58
:101F2000102FFCD7112FFAD70001000CDB6B010139
:101F30001E6B0001DC6B01011F6B0001DD91DD9365
:101F4000896B0101206BEA6A8A0EE96E06010F6B4C
:101F5000116B400E106F0001DADFEA6ADE0EE96EE7
:101F600006010F6B116B510E106F0001D0DF15EFE2
:101F700058F0040EEA6ECC0EE96EEF500DE00A0E3A
:101F8000016E006A002EFED7012EFBD75F0E006E99
:101F9000002EFED7EF2EF3D7000C0401D3B102D0F0
:101FA0008C9801D08C889598D3B302D08C9A01D0AC
:101FB0008C8A959AD3B502D08C9C01D08C8C959C40
:101FC000D3B702D08C9E01D08C8E959E00008C845D
:101FD0009594050E006E002EFED78C94959400010A
:101FE000000C0401D46B9588000E83B8010ED41345
:101FF000958A000E83BA010E006ED890003600500C
:10200000D413958C000E83BC010E006E0036003692
:10201000FC0E00160050D413958E000E83BE010EE8
:10202000006E003600360036F80E00160050D4134D
:10203000D4C401F00001000C9588958A958C958E8A
:102040008C82959200008C8495940000CADF01C0B8
:10205000D3F48C94959400008C849594020E006EB9
:10206000002EFED70000BDDF01C0D2F48C94959401
:102070009598959A959C959E0401D339006EF00E23
:1020800000160050D211016E00014AEF10F08C9042
:102090009590D2D701C0D2F4040101AE02D0000164
:1020A000F8D7D05302E18C9001D08C80959000003D
:1020B0008C92959200008C949594D139D26F0F0E2A
:1020C000D217D2C4D3F4000168DF0401D1510F0B41
:1020D000D26FD36F000161DF000C9598959A959CA3
:1020E000959E9594959095928C9095908C929592C2
:1020F0008C9495940F0E0401CC6F00013ADF010E11
:102100000401826F825103080CE3030ED36F0001B8
:1021100044DF050E0401CC6F00012BDF0401822B8C
:10212000F1D7020ED36F000138DF0401826B8251B8
:10213000030813E3036A8251F2CF83F4F29E000195
:10214000D5EC03F0040183BFF28E836FD06BD16FA7
:1021500000019DDF0401822BEAD7000117EF58F040
:10216000080E016E0A0E006E002EFED78B96949616
:102170000B0E006E002EFED70401A4378B98D8B04A
:102180009488D8A09498948682A6FED7012E01D078
:1021900002D00001E7D70A0E006E002EFED78B9604
:1021A0009496000094880B0E006E002EFED70B0E46
:1021B000006E002EFED7948682A6FED7016A0B0E13
:1021C000006E002EFED782B801808B9694968B9875
:1021D00094980001000C94880A0E006E002EFED721
:1021E00094860B0E006E002EFED782A6FED78B982B
:1021F00094980A0E006E002EFED78B969496A1C47A
:10220000A4F4AEDFA2C4A4F4ABDFA3C4A4F4A8DF9B
:1022100094980000948682A6FED70A0E006E002EC7
:10222000FED700D0000094880A0E006E002EFED764
:10223000250E006E002EFED7000C080E0401A36FC1
:1022400000C0A4F494880B0E006E002EFED7948676
:1022500082A6FED782B8D88082A8D89001360A0E0E
:10226000006E002EFED794968B96A32FEBD7948802
:102270000B0E006E002EFED78B98A451D8A4949814
:102280000000948682A6FED70A0E006E002EFED7AE
:102290008B9694960B0E006E002EFED78B9894981A
:1022A0000001000C0401A16B94880A0E006E002E40
:1022B000FED794860B0E006E002EFED782A6FED7A8
:1022C0008B9894980A0E006E002EFED78B969496EB
:1022D0009FC4A4F4000144DFA0C4A4F441DF9488A7
:1022E0000A0E006E002EFED794860B0E006E002E96
:1022F000FED782A6FED78B9894980A0E006E002E09
:10230000FED78B96949604019F510109A26FA46F8A
:10231000000126DF006A91DF01C0A1F4949800005B
:10232000948682A6FED70A0E006E002EFED700D03D
:10233000000094880A0E006E002EFED7250E006E57
:10234000002EFED70401A1C401F00001000C04011D
:10235000826B400EA16F180EA26FFF0EA36F0001DB
:102360003ADF400E0401A16F190EA26F010EA36F98
:10237000000131DF400E0401A16F1A0EA26FA36BA2
:10238000000129DF400E0401A16F1B0EA26FA36B99
:10239000000121DF400E0401A16F1C0EA26FA36B90
:1023A000000119DF400E0401A16F200EA26FA36B84
:1023B000000111DF400E0401A16F210EA26FFE0E7D
:1023C000A36F000108DF400E0401A16F220EA26F6F
:1023D000FF0EA36F0001FFDE400E0401A16F230E6C
:1023E000A26FFF0EA36F0001F6DE400E0401A16F85
:1023F000240EA26FFF0EA36F0001EDDE400E04015C
:102400009F6FA06B00014EDF01C082F4400E0401FB
:102410009F6F010EA06F000145DF01C082F4400EE6
:102420000401A16F2A0EA26F030EA36F0001D3DE79
:10243000FF0E886F400E0401A16F0A0EA26F88C0C4
:10244000A3F40001C8DE25EF58F010C612F60FC63F
:1024500011F612C603F0060111C6E9FF12C6EAFF23
:10246000EF5206E0112BD8B4122B0001F2D706016F
:102470000F51115D006E10511259036E00C001F032
:102480000001000C0401CD2D01D003D0400ECE6F11
:1024900001D0CE6B010ECC5DCE27CE518009CF6F1F
:1024A000D06BD16F0001F3DD000C0401CB510C0A9D
:1024B000000105E0060A0FE0020A15E01BD0040146
:1024C000D06B010ED16F0001E2DD020E0401CC6F72
:1024D00000014FDD17D0010E0401CC6F020ECD6F4D
:1024E0000001D0DF0FD00401D06B100ED16F0001BE
:1024F000CEDD08D0010E0401D06FCBC4D1F40001B1
:10250000C6DD00D0000C0401C96BC8C410F6C7C4F6
:102510000FF600019ADF0152D8B48ED0C8C410F66D
:10252000C7C40FF692DF01500401C95DD8B085D051
:10253000036AC951C725E96EC8510320EA6EEF50FE
:10254000010A00010DE0030A26E0010A3FE0080A43
:1025500058E0070A5EE0060A5CE0020A5AE059D039
:102560000401C95317E1010ECC6FCD6F00018ADF62
:10257000200E0401CB6F000198DF010E0401CC6F27
:10258000020ECD6F00017EDF200E0401CB6F000133
:102590008CDF04014ED00401C95317E1010ECC6F4A
:1025A000CD6F00016FDF3E0E0401CB6F00017DDFB8
:1025B000010E0401CC6F020ECD6F000163DF200E0F
:1025C0000401CB6F000171DF040133D00401C95352
:1025D00017E1010ECC6FCD6F000154DF200E040116
:1025E000CB6F000162DF010E0401CC6F020ECD6FD4
:1025F000000148DF3E0E0401CB6F000156DF0401ED
:1026000018D0010E0401CC6FCD6F00013BDF040137
:1026100010D0036A0401C951C725E96EC8510320CF
:10262000EA6EEFCFCAF4CAC4CBF400013EDF040166
:1026300000D0C92B000172D704010001000C020177
:10264000206B1F6B20C222F21FC221F2010EEA6E24
:10265000210EE96E06010F6B116BFE0E106F00016B
:1026600056DCDD9751EF58F004019D533FE099C4CB
:10267000E9FF9AC4EAFFEFCF9EF49CC403F09BC429
:10268000E9FF9CC4EAFFEF509E5D17E09AC403F097
:1026900099C4E9FF9AC4EAFFEFCF9EF49CC403F00B
:1026A0009BC4E9FF9CC4EAFFEF509E5D02E2FF0E6F
:1026B00001D0010E016E1CD00BD09AC403F099C456
:1026C000E9FF9AC4EAFFEF5203E1000E016E10D059
:1026D0009AC403F09951992BD8B49A2B9CC403F057
:1026E0009B519B2BD8B49C2B9D07BFD7000E016E2E
:1026F0000001CAEF13F00401836B826B846B856B5E
:10270000200E866F876F886F896F8A6F8B6F8C6FD3
:102710008D6F8E6F8F6F906F916F926F936F946FBD
:10272000956F966F976F986B030E836FE00E826FB5
:10273000846B84510F0822E3F2CF99F4F29E83C494
:10274000AAFF82C4A9FFA69CA69EA680A85099BFF6
:10275000F28E856F010ECC6F00010BDC036A040161
:102760008451860FE96E040E0320EA6E85C4EFFFE4
:10277000010E8227000E8323842BDBD7966B040E79
:102780009A6F860E996F9C6B310E9B6F100E9D6F2A
:1027900000016AD7015204E1010E016E04D003D09A
:1027A000FF0E016E00D053EF58F00401886B060E47
:1027B0004D6E4E6A4F6A506A516A526A546A556A3F
:1027C000566A596A586A5B6A5A6A886B88510A085D
:1027D0000DE3D8908835036A5C0FE96E000E032084
:1027E000EA6EEC6AED52EF6A882BF0D7886B88515D
:1027F0000A080DE3D8908835036A720FE96E000E5F
:102800000320EA6EEC6AED52EF6A882BF0D70001E4
:1028100013EF14F00401836B826B856B846B866B02
:10282000876B0001C2D7AA6AA96A4DC0A8FFA69CFF
:10283000A69EA684F250006EF29E0F01550EA76E62
:10284000AA0EA76EA682A6B2FED7A6940050F212D8
:10285000AA6A010EA96E4EC0A8FFA69CA69EA684D9
:10286000F2CF00F0F29E550EA76EAA0EA76EA682BA
:10287000A6B2FED7A6940050F212AA6A020EA96E62
:1028800050C0A8FFA69CA69EA684F2CF00F0F29EA0
:10289000550EA76EAA0EA76EA682A6B2FED7A69464
:1028A0000050F212AA6A030EA96E51C0A8FFA69C9E
:1028B000A69EA684F2CF00F0F29E550EA76EAA0E39
:1028C000A76EA682A6B2FED7A6940050F212AA6AFC
:1028D000040EA96E52C0A8FFA69CA69EA684F2CFA5
:1028E00000F0F29E550EA76EAA0EA76EA682A6B2A3
:1028F000FED7A6940050F212AA6A050EA96E54C023
:10290000A8FFA69CA69EA684F2CF00F0F29E550ECC
:10291000A76EAA0EA76EA682A6B2FED7A6940050F6
:10292000F212AA6A060EA96E55C0A8FFA69CA69E22
:10293000A684F2CF00F0F29E550EA76EAA0EA76EE7
:10294000A682A6B2FED7A6940050F212AA6A070E7B
:10295000A96E56C0A8FFA69CA69EA684F2CF00F042
:10296000F29E550EA76EAA0EA76EA682A6B2FED73D
:10297000A6940050F2120401836B100E826F866BD6
:1029800086510A0858E3D8908635036A5C0FE96ED1
:10299000000E0320EA6EECCF89F4ED52EFCF88F4FD
:1029A00089C487F483C4AAFF82C4A9FF87C4A8FF8F
:1029B000A69CA69EA684F250006EF29E0F01550EB4
:1029C000A76EAA0EA76EA682A6B2FED7A694005046
:1029D000F212010E04018227000E8323D89086355F
:1029E000036A5C0FE96E000E0320EA6EECCF89F4F7
:1029F000ED52EFCF88F488C487F483C4AAFF82C461
:102A0000A9FF87C4A8FFA69CA69EA684F250006ECC
:102A1000F29E0F01550EA76EAA0EA76EA682A6B251
:102A2000FED7A6940050F212010E04018227000E78
:102A30008323862BA5D7836B260E826F866B8651E8
:102A40000A0858E3D8908635036A720FE96E000EC3
:102A50000320EA6EECCF89F4ED52EFCF88F489C4FD
:102A600087F483C4AAFF82C4A9FF87C4A8FFA69CD9
:102A7000A69EA684F250006EF29E0F01550EA76E20
:102A8000AA0EA76EA682A6B2FED7A6940050F21296
:102A9000010E04018227000E8323D8908635036A35
:102AA000720FE96E000E0320EA6EECCF89F4ED524E
:102AB000EFCF88F488C487F483C4AAFF82C4A9FF37
:102AC00087C4A8FFA69CA69EA684F250006EF29E24
:102AD0000F01550EA76EAA0EA76EA682A6B2FED74C
:102AE000A6940050F212010E04018227000E8323E7
:102AF000862BA5D7030E836FE00E826F866B8651FF
:102B00000F0827E3036A8651310FE96E000E032098
:102B1000EA6EEFCF87F483C4AAFF82C4A9FF87C4FB
:102B2000A8FFA69CA69EA684F250006EF29E0F01FE
:102B3000550EA76EAA0EA76EA682A6B2FED7A694C1
:102B40000050F212010E04018227000E8323862B0F
:102B5000D6D7030E836FF00E826F856B846B866B06
:102B60008651110849E3036A86511F0FE96E000E72
:102B70000320EA6EEFCF88F488512F0803E28851D2
:102B8000390802E2000E01D0010E010833E185533D
:102B900031E1845105082EE3036A86511F0FE96E67
:102BA000000E0320EA6EEFCF87F483C4AAFF82C42D
:102BB000A9FF87C4A8FFA69CA69EA684F250006E1B
:102BC000F29E0F01550EA76EAA0EA76EA682A6B2A0
:102BD000FED7A6940050F212050E0401CC6F00013E
:102BE000B9EC0FF00401842BD8B4852B010E822799
:102BF000000E8323862BB4D7030E836FF60E826FED
:102C0000866B8651080835E3036A8651430FE96EE7
:102C1000000E0320EA6EEFCF87F483C4AAFF82C4BC
:102C2000A9FF87C4A8FFA69CA69EA684F250006EAA
:102C3000F29E0F01550EA76EAA0EA76EA682A6B22F
:102C4000FED7A6940050F212F2CF88F4F29E83C40D
:102C5000AAFF82C4A9FFA69CA69EA680A850040134
:102C600088BFF28E876F010E8227000E8323862B8A
:102C7000C8D7000158EF58F0596A586A5B6A5A6A17
:102C80005150060829E25150110826E3070E515C05
:102C9000006ED89000360050036A5C0FE96E000E9B
:102CA0000320EA6EECCF03F0ED52EFCF58F003C0F3
:102CB00059F0070E515C006ED89000360050036A40
:102CC000720FE96E000E0320EA6EECCF03F0ED52B6
:102CD000EFCF5AF003C05BF05550060829E255507B
:102CE000110826E3070E555C006ED89000360050A0
:102CF000036A5C0FE96E000E0320EA6EECCF03F06E
:102D0000ED52EFCF58F003C059F0070E555C006E3E
:102D1000D89000360050036A720FE96E000E03204F
:102D2000EA6EECCF03F0ED52EFCF5AF003C05BF048
:102D3000000C016A026A006A036A0601155102E189
:102D4000145118E0100E166FD89012371337003652
:102D500003361551035C02E11451005C07E3145182
:102D6000005ED8A003061551035ED88001360236F6
:102D7000162FEAD70001000CD89002011F35026E11
:102D80002035036E0250210FE96E010E0320EA6E1A
:102D9000EC6AED520FC6EFFF010E1F250601106F02
:102DA000000E020120210601116F136F10C612F6EA
:102DB000156B7F0E146F0001BCDF00C01FF2020113
:102DC00003C020F20001DD87000C0401C46BC36B5B
:102DD000C56BF2CFC6F4F29EAA6AA96AA69CA69E0B
:102DE000A680A850C6BFF28E4D6EF2CFC6F4F29EFA
:102DF000AA6A010EA96EA69CA69EA680A850C6BF70
:102E0000F28E4E6EF2CFC6F4F29EAA6A020EA96E40
:102E1000A69CA69EA680A850C6BFF28E506EF2CF8A
:102E2000C6F4F29EAA6A030EA96EA69CA69EA68070
:102E3000A850C6BFF28E516EF2CFC6F4F29EAA6AB7
:102E4000040EA96EA69CA69EA680A850C6BFF28EB0
:102E5000526EF2CFC6F4F29EAA6A050EA96EA69C27
:102E6000A69EA680A850C6BFF28E546EF2CFC6F4BE
:102E7000F29EAA6A060EA96EA69CA69EA680A850DF
:102E8000C6BFF28E556EF2CFC6F4F29EAA6A070E46
:102E9000A96EA69CA69EA680A850C6BFF28E566EAE
:102EA000C46B100EC36FC56BC5510A0833E3F2CF74
:102EB000C6F4F29EC4C4AAFFC3C4A9FFA69CA69EE2
:102EC000A680A850C6BFF28EC16F010EC327000EA8
:102ED000C423F2CFC6F4F29EC4C4AAFFC3C4A9FFA0
:102EE000A69CA69EA680A850C6BFF28EC26F010EF9
:102EF000C327000EC423D890C535036A5C0FE96E62
:102F0000000E0320EA6EC1C4ECFFED52C2C4EFFF15
:102F1000C52BCAD7C46B260EC36FC56BC5510A0833
:102F200033E3F2CFC6F4F29EC4C4AAFFC3C4A9FF20
:102F3000A69CA69EA680A850C6BFF28EC16F010EA9
:102F4000C327000EC423F2CFC6F4F29EC4C4AAFF66
:102F5000C3C4A9FFA69CA69EA680A850C6BFF28E99
:102F6000C26F010EC327000EC423D890C535036A73
:102F7000720FE96E000E0320EA6EC1C4ECFFED5241
:102F8000C2C4EFFFC52BCAD7000176DE4F6A4DA23F
:102F900006D0160E06010F6F0001EEDE05D0170EEB
:102FA00006010F6F0001E8DE000C04019951010ACF
:102FB00000010DE0030AD8B4A2D0010AD8B403D1AD
:102FC000070AD8B464D1040AD8B403D202D2020EDC
:102FD000EA6E2F0EE96EF2CF9AF4F29E000EB0EC7C
:102FE00007F00A000900F550EE6E0009FBE104014C
:102FF0009ABFF28E020EEA6E410EE96EF2CF9AF49B
:10300000F29E000E0001C8EC07F00A000900F5501E
:10301000EE6E0009FBE104019ABFF28E020EEA6E29
:10302000530EE96EF2CF9AF4F29E000E0001E0EC2E
:1030300007F00A000900F550EE6E0009FBE10401FB
:103040009ABFF28E020EEA6E650EE96EF2CF9AF426
:10305000F29E000E0001F8EC07F00A000900F5509E
:10306000EE6E0009FBE104019ABFF28E020EEA6ED9
:10307000770EE96EF2CF9AF4F29E000E000110EC8A
:1030800008F00A000900F550EE6E0009FBE10401AA
:103090009ABFF28E020EEA6E890EE96EF2CF9AF4B2
:1030A000F29E000E000128EC08F00A000900F5501D
:1030B000EE6E0009FBE104019ABFF28E010E0201DF
:1030C000AD6F1EB40AD0036AAD51B80FE96E020E9F
:1030D0000320EA6E040EEF6E09D0036AAD51B80FFB
:1030E000E96E020E0320EA6E050EEF6E036AAD5123
:1030F000BD0FE96E020E0320EA6EEF6AF7D1020EF1
:10310000EA6E2F0EE96EF2CF9AF4F29E000E40ECBA
:1031100008F00A000900F550EE6E0009FBE1040119
:103120009ABFF28E020EEA6E410EE96EF2CF9AF469
:10313000F29E000E000158EC08F00A000900F5505C
:10314000EE6E0009FBE104019ABFF28E020EEA6EF8
:10315000530EE96EF2CF9AF4F29E000E000170EC6D
:1031600008F00A000900F550EE6E0009FBE10401C9
:103170009ABFF28E020EEA6E650EE96EF2CF9AF4F5
:10318000F29E000E000188EC08F00A000900F550DC
:10319000EE6E0009FBE104019ABFF28E020E0201FD
:1031A000AD6F036AAD51B80FE96E020E0320EA6EEF
:1031B000030EEF6E036AAD51BD0FE96E020E0320E0
:1031C000EA6EEF6A93D1020EEA6E2F0EE96EF2CF2D
:1031D0009AF4F29E000EA0EC08F00A000900F550E7
:1031E000EE6E0009FBE104019ABFF28E020EEA6E58
:1031F000410EE96EF2CF9AF4F29E000E0001B8EC97
:1032000008F00A000900F550EE6E0009FBE1040128
:103210009ABFF28E020EEA6E530EE96EF2CF9AF466
:10322000F29E000E000170EC08F00A000900F55053
:10323000EE6E0009FBE104019ABFF28E020EEA6E07
:10324000650EE96EF2CF9AF4F29E000E000188EC52
:1032500008F00A000900F550EE6E0009FBE10401D8
:103260009ABFF28E030E0201AD6F036AAD51B80F23
:10327000E96E020E0320EA6E030EEF6E036AAD5193
:10328000BD0FE96E020E0320EA6EEF6A2FD1515096
:10329000060803E25150110806E25550060854E2B0
:1032A0005550110851E3020EEA6E2F0EE96EF2CF6F
:1032B0009AF4F29E000ED0EC08F00A000900F550D6
:1032C000EE6E0009FBE104019ABFF28E020EEA6E77
:1032D000410EE96EF2CF9AF4F29E000E0001E8EC86
:1032E00008F00A000900F550EE6E0009FBE1040148
:1032F0009ABFF28E020EEA6E530EE96EF2CF9AF486
:10330000F29E000E000100EC09F00A000900F550E1
:10331000EE6E0009FBE104019ABFF28E040E020179
:10332000AD6F036AAD51B80FE96E020E0320EA6E6D
:10333000020EEF6E036AAD51BD0FE96E020E03205F
:10334000EA6EEF6A45D00001020EEA6E2F0EE96EBA
:10335000F2CF9AF4F29E000ED0EC08F00A000900B9
:10336000F550EE6E0009FBE104019ABFF28E020EE9
:10337000EA6E410EE96EF2CF9AF4F29E000E000161
:1033800018EC09F00A000900F550EE6E0009FBE1A7
:1033900004019ABFF28E050E0201AD6F036AAD51B2
:1033A000B80FE96E020E0320EA6EEF6A036AAD51B0
:1033B000BD0FE96E020E0320EA6EEF6A04013F6B57
:1033C0003E6B3D6B3C6B3DC441F43CC440F4020198
:1033D0008DD0020EEA6E2F0EE96EE26A310EE16EBA
:1033E000E752E6CFEEFFFCE1020EEA6E410EE96E17
:1033F000E26A1F0EE16EE752E6CFEEFFFCE1020E3D
:10340000EA6E530EE96EF2CF9AF4F29E000E30ECA3
:1034100009F00A000900F550EE6E0009FBE1040115
:103420009ABFF28E020EEA6E650EE96EF2CF9AF442
:10343000F29E000E000148EC09F00A000900F55068
:10344000EE6E0009FBE104019ABFF28E020EEA6EF5
:10345000770EE96EF2CF9AF4F29E000E000160EC56
:1034600009F00A000900F550EE6E0009FBE10401C5
:103470009ABFF28E020EEA6E890EE96EF2CF9AF4CE
:10348000F29E000E000178EC09F00A000900F550E8
:10349000EE6E0009FBE104019ABFF28E020EEA6EA5
:1034A0009B0EE96EF2CF9AF4F29E000E000190ECB2
:1034B00009F00A000900F550EE6E0009FBE1040175
:1034C0009ABFF28E0201AD6B036AAD51B80FE96E7F
:1034D000020E0320EA6E050EEF6E036AAD51BD0FBA
:1034E000E96E020E0320EA6EEF6A00D00001000CC4
:1034F000C8C4CDF4C7C4CCF40401CB5324E0CAC47F
:1035000003F0C9C4E9FFCAC4EAFFEF521CE0CDC40E
:1035100003F0CC51CC2BD8B4CD2BCE6F03C0CFF45D
:10352000CAC403F0C951C92BD8B4CA2BE96E03C071
:10353000EAFFEFCFD0F4CFC4EAFFCEC4E9FFD0C496
:10354000EFFFCB07DAD7CB530CE0CDC403F0CC515F
:10355000CC2BD8B4CD2BE96E03C0EAFFEF6ACB07C2
:10356000F2D7C7C401F0C8C402F00001000C040E79
:10357000EA6E9C0EE96E06010F6B116B130E106F55
:10358000000187EC0FF0040EEA6EAF0EE96E060143
:103590000F6B116B130E106F000187EC0FF004011D
:1035A0009A51120DF350036A2F0F016E020E03227F
:1035B00001C0C2F403C0C3F4040EC86F9C0EC76FF1
:1035C00003C0CAF401C0C9F4120ECB6F000190DF32
:1035D0000C0E04019C6F036A0201AD51AE0FE96E3F
:1035E000020E0320EA6EEF2C03D03E0E04019D6F05
:1035F000040E0401C86F9C0EC76F000183EC12F02B
:10360000050E0401CC6F0001B9EC0FF004019B51D1
:10361000120DF350036A2F0F016E020E032201C038
:10362000C2F403C0C3F4040EC86FAF0EC76F03C06B
:10363000CAF401C0C9F4120ECB6F000159DF0A0EA3
:103640000401AF6F036A0201AD51AE0FE96E020EC5
:103650000320EA6EEF50020803E13E0E0401B06F52
:10366000040E0401C86FAF0EC76F000183EC12F0A7
:10367000000C036A0201AD51AE0FE96E020E032089
:10368000EA6EEF5002081DE1036AAD51B30FE96E17
:10369000020E0320EA6E010EEF5C0401846F036AE0
:1036A0000201AD51B30FE96E020E0320EA6EEFCFB7
:1036B00085F484C49AF485C49BF4000158DF1AD0C1
:1036C0000201036AAD51B30FE96E020E0320EA6EE8
:1036D000EFCF84F4036AAD51B30FE96E020E0320FD
:1036E000EA6E010EEF240401856F84C49AF49B6F87
:1036F00000013DDF000C0401AA6B0001DDA318D01E
:10370000036A01011F51DE0FE96E000E0320EA6E0D
:10371000EFCFAAF40401010E01011F25500802E2B7
:103720001F6B01D01F2B1E511F5D03E10001DD93B4
:1037300001010401AAC401F00001000C0401A96BFD
:103740000001DDA304D0D7DF01C0A9F4FAD7000C33
:103750000900F6CF2BF5F7CF2CF5F8CF2DF5F55066
:103760009EA8FED7AD6E2BC5F6FF2CC5F7FF2DC565
:10377000F8FF05012A2F01D002D00001E9D700018E
:10378000000C05013051016A2F5D03E22FC500F0E6
:103790000CD0006A080E316F2F3700363051005CB4
:1037A000D8B0006E0136312FF7D70001000C200E83
:1037B000040191A9300E926F90C400F090AF07D031
:1037C000001E002A00C090F42D0E926F918F0150C0
:1037D00090C42FF5640E0501306F0001D2DF00C0E8
:1037E00090F4300E01240401936F90C42FF50A0E5B
:1037F0000501306F0001C5DF300E00240401956F14
:10380000300E0124946F92C400F091A702D091AFC2
:10381000919591B90BD091AF22D091B520D000C035
:1038200093F491B31CD000C094F419D0300E935D82
:1038300016E100C093F4200E926F91A704D09195E9
:10384000918391AF9193300E945D09E100C094F49F
:10385000200E936F91A7F7D7919391AF919191A576
:1038600004D092519EA8FED7AD6E91A304D093517F
:103870009EA8FED7AD6E91A104D094519EA8FED70C
:10388000AD6E95519EA8FED7AD6E000196EF1DF06E
:103890000401AEBF10D00F0E006EAD3900160A0E37
:1038A000005C03E2300E002602D0AE51002600502C
:1038B0009EA8FED7AD6E0F0EAD170A0EAD5D02E2EB
:1038C000300E02D0AE9FAE51AD27AD519EA8FED7AF
:1038D000AD6E0001000C0701FF5108010103F3CF99
:1038E00001F0F4CF00F00203F35000260051010371
:1038F000F3500020026E0001000CEACFB7F4E9CFCC
:10390000B6F40401B039F009B26FB227E20FB36F19
:10391000320FB56FB0510F0BB327B327B527E90F9F
:10392000B46FB427B427AF390F0BB427B527B4371A
:10393000B537B51FB537AF510F0BB527B237070EE7
:10394000B16F0A0EB407B527FDE3B307B427FDE353
:10395000B207B327FDE3B107B227FDE3040EEA6E19
:10396000B10EE96E070EB615B69DE926B50EE95CF7
:10397000D8B4B68DEF50006E08E1B6BD06D0B6B92A
:103980000CD0B6B702D0200E03D0B687B699300E51
:10399000002600509EA8FED7AD6EEE50B6ADE6D71D
:1039A0000001000C0401AA6BA96B130EAC6F880E0A
:1039B000AB6F0001DDB342D0AAC400F8A9C4FFF781
:1039C0000801026B0A0E016F000185DF02C0AEF430
:1039D00001C0ADF40401AC51025C25E303E1AB513D
:1039E000AD5D21E34DA01ED00A0EF66E1D0EF76EE2
:1039F000000EF86E1E0E05012A6F0001A9DE100EE2
:103A0000E96EACC4B0F4ABC4AFF477DF2B0EF66E46
:103A10001D0EF76E000EF86E050E05012A6F0001EF
:103A200097DE04013FD00A0ECC6F0001B9EC0FF015
:103A30000401A92BD8B4AA2BBCD700014DA02BD0D0
:103A4000AAC400F8A9C4FFF70801026B0A0E016FAF
:103A5000000141DF02C0AEF401C0ADF4320EF66EDB
:103A60001D0EF76E000EF86E240E05012A6F000180
:103A70006FDE100EE96EAEC4B0F4ADC4AFF43DDF3E
:103A8000590EF66E1D0EF76E000EF86E050E05014E
:103A90002A6F00015DDE050E0401CC6F0001B9EC58
:103AA0000FF004010001000C49DE89C48CF488C4C5
:103AB0008DF48BC48EF48AC48FF4800EA4A8FED734
:103AC0006D6E040EA4A8FED76D6E04018C51A4A8DF
:103AD000FED76D6E8D51A4A8FED76D6E8E51A4A831
:103AE000FED76D6E8F51A4A8FED76D6EFF0EA4A8F1
:103AF000FED76D6E4DA076D089C48CF488C48DF449
:103B00008BC48EF48AC48FF4CC0EF66E1D0EF76E45
:103B1000000EF86E080E05012A6F000119DE87C439
:103B200090F41F0E0401916F000141D6D60EF66E7F
:103B30001D0EF76E000EF86E0C0E05012A6F0001C7
:103B400007DE800E0401AD6F570EAE6F0001A0DEE0
:103B5000200E9EA8FED7AD6E040E0401AD6F570E69
:103B6000AE6F000195DE200E9EA8FED7AD6E8CC410
:103B7000ADF4570E0401AE6F00018ADE200E9EA840
:103B8000FED7AD6E8DC4ADF4570E0401AE6F0001CB
:103B90007FDE200E9EA8FED7AD6E8EC4ADF4570E0C
:103BA0000401AE6F000174DE200E9EA8FED7AD6E3C
:103BB0008FC4ADF4570E0401AE6F000169DE200E14
:103BC0009EA8FED7AD6EFF0E0401AD6F570EAE6F0F
:103BD00000015EDE0A0E9EA8FED7AD6E0D0E9EA8F9
:103BE000FED7AD6E0001DEDE000CDD99DD9BDD9DB4
:103BF00004013D6B3C6B3DC441F43CC440F441C402
:103C00003FF440C43EF4FF0E3D6F3C6F000131DDD8
:103C10000201AD51040812E10001DDAF0ED0DD9FBD
:103C2000010E0401876F59C089F458C088F45BC045
:103C30008BF45AC08AF4000137DF02010001000C46
:103C4000DDB95ED00201AD51000A000107E0020AB1
:103C500029E0010A27E0020A25E024D0036A0201D4
:103C6000AD51AE0FE96E020E0320EA6EEF6A036AF1
:103C7000AD51B30F016E020E0322040103C085F49F
:103C8000036A0201AD51BD0FE96E020E0320EA6E18
:103C9000EFCF86F4040185C4EAFF01C0E9FF86C4C2
:103CA000EFFF2BD00201AD6BADC299F40001D5EC52
:103CB00017F0036A0201AD51AE0FE96E020E032048
:103CC000EA6EEF6A036AAD51B30F016E020E032272
:103CD000040103C085F4036A0201AD51BD0FE96E12
:103CE000020E0320EA6EEFCF86F4040185C4EAFFDA
:103CF00001C0E9FF86C4EFFF00D00001BADC01D0AB
:103D000074DF000C0401826B826B8251020821E394
:103D1000036A8251AE0FE96E020E0320EA6EEF6A6B
:103D2000036A8251B30F016E020E032203C084F4B2
:103D3000036A8251BD0FE96E020E0320EA6EEFCFD7
:103D400085F484C4EAFF01C0E9FF85C4EFFF822B3C
:103D5000DCD70201AD6B0001DD99DD9BDD9D040127
:103D60003D6B3C6B3DC441F43CC440F441C43FF462
:103D700040C43EF4020EEA6E2F0EE96EE26A310E86
:103D8000E16EE752E6CFEEFFFCE1020EEA6E410E75
:103D9000E96EE26A1F0EE16EE752E6CFEEFFFCE14C
:103DA00000014EDF73EF58F004018F6B8E6B8D5363
:103DB00002E1010E8D6F94880A0E006E002EFED770
:103DC00094860B0E006E002EFED782A6FED78B982F
:103DD00094980A0E006E002EFED78B96949689C496
:103DE000A4F40001B0EC10F004018A518009906F36
:103DF000A46F0001B0EC10F094880A0E006E002E43
:103E0000FED794860B0E006E002EFED782A6FED73C
:103E10008B9894980A0E006E002EFED78B9694967F
:103E2000040189510109906FA46F0001B0EC10F0FA
:103E300004018F6B8E6B010E8D5D8F5314E18E5DCF
:103E400012E28B518E25E96E8C518F21EA6E010EA4
:103E5000006E00011DEC11F001C0EFFF04018E2B7C
:103E6000D8B48F2BE8D7010E8D5D036A8B25E96EE0
:103E70008C510320EA6E006A00011DEC11F001C0B4
:103E8000EFFF94980000948682A6FED70A0E006E7B
:103E9000002EFED700D0000094880A0E006E002E7F
:103EA000FED7250E006E002EFED704018BC4E9FF5D
:103EB0008CC4EAFFEFCF01F0000176EF1FF00401A0
:103EC000826B836B846B856B866B876B8881938039
:103ED00081A001D04CD1400E896F8A6B040E8C6F8B
:103EE000820E8B6F020E8D6F00015ED701C082F4CF
:103EF000FF0E0401821B831B010E83174DA01ED0F1
:103F0000E00EF66E190EF76E000EF86E120E050139
:103F10002A6F00011DDC83C4ADF4370E0401AE6FBF
:103F20000001B6DC200E9EA8FED7AD6E82C4ADF4B3
:103F3000370E0401AE6F0001ABDC0401825303E1D4
:103F4000835301E114D184A804D0822D01D001D083
:103F50000ED18251000A000111E0010A10E0030AAB
:103F600015E0060A1AE00C0A1FE0180A24E0300ADD
:103F700029E0600A2EE0C00A33E039D093D0010E68
:103F800006010F6F0001BCEC16F08CD00B0E060181
:103F90000F6F0001BCEC16F085D00E0E06010F6FFE
:103FA0000001BCEC16F07ED0030E06010F6F00017D
:103FB000BCEC16F077D00D0E06010F6F0001BCECC3
:103FC00016F070D00C0E06010F6F0001BCEC16F05D
:103FD00069D0050E06010F6F0001BCEC16F062D02F
:103FE000090E06010F6F0001BCEC16F05BD0040156
:103FF00088914DA055D0FA0EF66E190EF76E000E90
:10400000F86E160E05012A6F0001A8EC1BF083C4A0
:10401000ADF4370E0401AE6F00013ADC200E9EA80D
:10402000FED7AD6E5B0E9EA8FED7AD6E82C4ADF41A
:10403000370E0401AE6F00012BDC5D0E9EA8FED78B
:10404000AD6E04018351FF0A896F8251FF0A8A6FA6
:104050001A0EF66E1A0EF76E000EF86E160E0501A9
:104060002A6F0001A8EC1BF089C4ADF4370E0401DF
:10407000AE6F00010DDC200E9EA8FED7AD6E5B0E6C
:104080009EA8FED7AD6E8AC4ADF4370E0401AE6FA4
:10409000000148EC1CF05D0E9EA8FED7AD6E040139
:1040A00066D0000104018351000A000103E0010A07
:1040B00002E008D05CD0070E06010F6F0001BCECD7
:1040C00016F055D0040188914DA050D03A0EF66EEE
:1040D0001A0EF76E000EF86E170E05012A6F00011A
:1040E000A8EC1BF083C4ADF4370E0401AE6F0001E1
:1040F00048EC1CF05D0E9EA8FED7AD6E200E9EA86B
:10410000FED7AD6E82C4ADF4370E0401AE6F000170
:1041100048EC1CF004018351FF0A896F8251FF0AA9
:104120008A6F5A0EF66E1A0EF76E000EF86E170EA4
:1041300005012A6F0001A8EC1BF089C4ADF4370E0D
:104140000401AE6F000148EC1CF05D0E9EA8FED786
:10415000AD6E200E9EA8FED7AD6E8AC4ADF4370EAC
:104160000401AE6F000148EC1CF0040100D0000116
:10417000BBEF20F0A4D675EF58F0DDA731D0D89072
:1041800002012135026E2235036E0250210FE96EC5
:10419000010E0320EA6EEFCF83F40401010E020149
:1041A00021250401846F000E020122210401856F84
:1041B000E8CF13F684C412F60601156B7F0E146F58
:1041C000000199EC16F000C021F2020103C022F2B6
:1041D0001F51215D06E12051225D03E10001DD97C1
:1041E0000201040183C401F0000133EF4CF00150DF
:1041F0009FC42FF5640E0501306F0001C1EC1BF068
:1042000000C09FF40150300E08E10401A0A30ED0BD
:10421000A0B70CD0A0B9200E04D00401A097A0999B
:10422000A081012601509EA8FED7AD6E9FC42FF538
:104230000A0E0501306F0001C1EC1BF000C09FF4B5
:104240000150300E08E10401A0B70BD0A0A109D0A5
:10425000A0B9200E0001012601509EA8FED7AD6E28
:104260000401300E9F279F519EA8FED7AD6E00011E
:10427000000C010E04019F5DDF0FD8B0B5D0210FF7
:104280000001F6EF21F00401A05303E18D98969808
:1042900002D08D889698A8D00401A05338E19F5190
:1042A000030804E10001889D30D004019F510508F6
:1042B00004E10001889329D004019F51090804E119
:1042C0000001889122D004019F51070804E10001F8
:1042D000889F1BD004019F510B0804E100018899BD
:1042E00014D004019F510E0804E1000188970DD0FD
:1042F00004019F510D0804E10001889B06D00401D0
:104300009F510C0803E100018895040137D09F51AB
:10431000030804E10001888D30D004019F51050895
:1043200004E10001888329D004019F51090804E1B8
:104330000001888122D004019F51070804E1000197
:10434000888F1BD004019F510B0804E1000188896C
:1043500014D004019F510E0804E1000188870DD09C
:1043600004019F510D0804E10001888B06D004016F
:104370009F510C0803E1000188850401400EA16FE4
:104380000A0EA26F88C0A3F40001EBEC10F0040148
:104390002BD0C00E8817400E0401A16F0A0EA26F29
:1043A00088C0A3F40001EBEC10F004011DD0030E53
:1043B0008817400E0401A16F0A0EA26F88C0A3F4F3
:1043C0000001EBEC10F004010FD0FF0E886F400EDF
:1043D0000401A16F0A0EA26F88C0A3F40001EBECE8
:1043E00010F0040101D004010001000CF2CF0DF027
:1043F000F29EE824F76AF736170FF66E440EF7229E
:10440000000EF86EFB6E0A00F550FA6E0800F550CB
:104410000DBEF28EF96E864286429842E64398427D
:10442000E6439842E6439842E643984298429842CF
:104430009842E643E643E643E643E643E643E64383
:10444000E643E643E643E643E643E643E643E64324
:10445000E6439243AE43CA43DDB92AD0040EEA6E66
:10446000A10EE96E06010F6B116B130E106F0001A8
:1044700087EC0FF0040E0401C86FA10EC76F020E87
:10448000CA6F2F0EC96F120ECB6F000178EC1AF0B5
:104490000C0E0401A16F040EC86FA10EC76F0001BE
:1044A00083EC12F0050E0401CC6F0001B9EC0FF0A3
:1044B000040EEA6EB40EE96E06010F6B116B130E5B
:1044C000106F000187EC0FF0040E0401C86FB40EEA
:1044D000C76FA0C4CAF49FC4C9F4120ECB6F000109
:1044E00078EC1AF00A0E0401B46F040EC86FB40E13
:1044F000C76F000183EC12F0000C0401A76BA153FD
:1045000007E1A25305E1A06BA46BA36BA66BA56B9F
:10451000A151770803E1770EA76F12D0D890A1358B
:10452000A96BA86F010EA825016E000EA921036ECC
:104530000150420FE96E040E0320EA6EEFCFA7F49C
:1045400000019EEC1BF0A4C4A8F4A3C4A9F4A6C463
:10455000AAF4A5C4ABF4800EA4A8FED76D6E020E1B
:10456000A4A8FED76D6E0401A051A4A8FED76D6E5D
:10457000A751A4A8FED76D6EA251A4A8FED76D6E58
:10458000A851A4A8FED76D6EA951A4A8FED76D6E40
:10459000AA51A4A8FED76D6EAB51A4A8FED76D6E2C
:1045A000FF0EA4A8FED76D6E4DA090D0A4C4A8F4B1
:1045B000A3C4A9F4A6C4AAF4A5C4ABF4960EF66EDF
:1045C0001D0EF76E000EF86E0C0E05012A6F00012D
:1045D000A8EC1BF0800E0401AD6F570EAE6F00010A
:1045E00048EC1CF0200E9EA8FED7AD6E020E040112
:1045F000AD6F570EAE6F000148EC1CF0200E9EA868
:10460000FED7AD6EA0C4ADF4570E0401AE6F00012D
:1046100048EC1CF0200E9EA8FED7AD6EA7C4ADF4EA
:10462000570E0401AE6F000148EC1CF0200E9EA84E
:10463000FED7AD6EA2C4ADF4570E0401AE6F0001FB
:1046400048EC1CF0200E9EA8FED7AD6EA8C4ADF4B9
:10465000570E0401AE6F000148EC1CF0200E9EA81E
:10466000FED7AD6EA9C4ADF4570E0401AE6F0001C4
:1046700048EC1CF0200E9EA8FED7AD6EAAC4ADF487
:10468000570E0401AE6F000148EC1CF0200E9EA8EE
:10469000FED7AD6EABC4ADF4570E0401AE6F000192
:1046A00048EC1CF0200E9EA8FED7AD6EFF0E040154
:1046B000AD6F570EAE6F000148EC1CF00A0E9EA8BD
:1046C000FED7AD6E0D0E9EA8FED7AD6E0001D2ECEA
:1046D0001CF0000C0401A76BA86BA15307E1A253C7
:1046E00005E1A06BA46BA36BA66BA56BD890A0355E
:1046F000AA6BA96F420EA925E96E040EAA21EA6EE3
:10470000EFCFA7F4A151770803E1770EA86F12D07D
:10471000D890A135AA6BA96F010EA925016E000ED4
:10472000AA21036E0150420FE96E040E0320EA6EC7
:10473000EFCFA8F400019EEC1BF0A4C4A9F4A3C41D
:10474000AAF4A6C4ABF4A5C4ACF4800EA4A8FED70A
:104750006D6E010EA4A8FED76D6E0401A751A4A82A
:10476000FED76D6EA851A4A8FED76D6EA251A4A865
:10477000FED76D6EA951A4A8FED76D6EAA51A4A84C
:10478000FED76D6EAB51A4A8FED76D6EAC51A4A838
:10479000FED76D6EFF0EA4A8FED76D6E4DA090D013
:1047A000A4C4A9F4A3C4AAF4A6C4ABF4A5C4ACF4ED
:1047B000600EF66E1D0EF76E000EF86E0C0E050103
:1047C0002A6F0001A8EC1BF0800E0401AD6F570E9C
:1047D000AE6F000148EC1CF0200E9EA8FED7AD6E17
:1047E000010E0401AD6F570EAE6F000148EC1CF0D6
:1047F000200E9EA8FED7AD6EA7C4ADF4570E0401DF
:10480000AE6F000148EC1CF0200E9EA8FED7AD6EE6
:10481000A8C4ADF4570E0401AE6F000148EC1CF0C3
:10482000200E9EA8FED7AD6EA2C4ADF4570E0401B3
:10483000AE6F000148EC1CF0200E9EA8FED7AD6EB6
:10484000A9C4ADF4570E0401AE6F000148EC1CF092
:10485000200E9EA8FED7AD6EAAC4ADF4570E04017B
:10486000AE6F000148EC1CF0200E9EA8FED7AD6E86
:10487000ABC4ADF4570E0401AE6F000148EC1CF060
:10488000200E9EA8FED7AD6EACC4ADF4570E040149
:10489000AE6F000148EC1CF0200E9EA8FED7AD6E56
:1048A000FF0E0401AD6F570EAE6F000148EC1CF017
:1048B0000A0E9EA8FED7AD6E0D0E9EA8FED7AD6E59
:1048C0000001D2EC1CF0000C0401856B846B876B3B
:1048D000866B9C6B9D6B9E6B4DA02CD0720EF66E02
:1048E0001C0EF76E000EF86E050E05012A6F000112
:1048F000A8EC1BF083C4ADF4570E0401AE6F0001A9
:1049000048EC1CF02F0E9EA8FED7AD6E83C49FF41A
:104910001B0E0401A06F00016ADC7D0EF66E1C0EFA
:10492000F76E000EF86E090E05012A6F0001A8EC63
:104930001BF00401010E835DF60FD8B067EF29F07C
:104940000A0F00016AEF29F084B852D00401832DC8
:104950002FD0400E9F6FA06B000152EC11F001C0F0
:104960009DF404019D51FE0815E19C511A0801E2D5
:1049700011D03C0ECC6F0001B9EC0FF004019C2B60
:10498000400E9F6FA06B000152EC11F001C09DF42E
:10499000E8D70401400E9F6FA06B000152EC11F0AC
:1049A00001C09DF404019D51FE0802E067EF29F06B
:1049B00083C49FF4010EA06F00015BDC040EEA6E5D
:1049C000880EE96EF2CF9FF4F29E000ED7EC06F04F
:1049D0000A000900F550EE6E0009FBE104019FBFDB
:1049E000F28E190E06010F6F0001BCEC16F01AD002
:1049F00083C49FF40401A06B00013BDC040EEA6E4B
:104A0000880EE96EF2CF9FF4F29E000EEFEC06F0F6
:104A10000A000900F550EE6E0009FBE104019FBF9A
:104A2000F28EFF00040E0401A06F880E9F6F00013C
:104A300013DD040167EF29F01EB0C3D084B8A3D002
:104A400004019E6B4DA608D05250020805E2525058
:104A50000A0802E3400E9E6F505202E0515202E1FA
:104A6000525268E0030E9F6FA06B000102DC050E3E
:104A700004019F6F010EA06F000139EC21F051522B
:104A800008E0070E04019F6FA06B000139EC21F0D4
:104A900008D0070E04019F6F010EA06F000139ECD2
:104AA00021F0525208E0090E04019F6FA06B000133
:104AB00039EC21F008D0090E04019F6F010EA06FA0
:104AC000000139EC21F0515214E0525212E0050E6F
:104AD00004019F6F010EA06F000139EC21F0040169
:104AE000A06BA16BA26BA46BA36BA66BA56B000163
:104AF00004DD3CEC16F0515208E059C085F458C072
:104B000084F45BC087F45AC086F4525004019E11AD
:104B10009F6F50C0A0F451C0A1F4A26F85C4A4F44B
:104B200084C4A3F487C4A6F486C4A5F40001D2DD2E
:104B30002AD00401030E9F6F010EA06F000139EC13
:104B400021F0050E04019F6F010EA06F000139ECEA
:104B500021F0070E04019F6F010EA06F000139ECD8
:104B600021F0090E04019F6F010EA06F000139ECC6
:104B700021F00401A06BA16BA26BA46BA36BA66BCD
:104B8000A56B0001A7DD0401835103081BE1040E9E
:104B9000EA6E880EE96EF2CF9FF4F29E000E0001DD
:104BA00007EC07F00A000900F550EE6E0009FBE182
:104BB00004019FBFF28E040EA06F880E9F6F00014C
:104BC0004BDC040167EF29F01EB0C6D084B8A5D035
:104BD00004019E6B4DA608D05650020805E25650BF
:104BE0000A0802E3400E9E6F545202E0555202E161
:104BF000565269E0050E9F6FA06B000139EC21F061
:104C0000030E04019F6F010EA06F000139EC21F02B
:104C1000555208E0070E04019F6FA06B000139ECAC
:104C200021F008D0070E04019F6F010EA06F000154
:104C300039EC21F0565208E0090E04019F6FA06B79
:104C4000000139EC21F008D0090E04019F6F010E1C
:104C5000A06F000139EC21F0555214E0565212E0D9
:104C6000030E04019F6F010EA06F000139EC21F0CB
:104C70000401A06BA16BA26BA46BA36BA66BA56BCD
:104C8000000128DD3CEC16F0555208E059C085F4CF
:104C900058C084F45BC087F45AC086F456500401AF
:104CA0009E119F6F54C0A0F455C0A1F4A26F85C49B
:104CB000A4F484C4A3F487C4A6F486C4A5F40001B4
:104CC0001CDC2BD00401030E9F6F010EA06F0001AE
:104CD00039EC21F0050E04019F6F010EA06F000159
:104CE00039EC21F0070E04019F6F010EA06F000147
:104CF00039EC21F0090E04019F6F010EA06F000135
:104D000039EC21F00401A06BA16BA26BA46BA36B27
:104D1000A66BA56B00017DEC22F004018351050810
:104D20001CE1040EEA6E880EE96EF2CF9FF4F29E4B
:104D3000000E00011FEC07F00A000900F550EE6EAE
:104D40000009FBE104019FBFF28E040EA06F880EE4
:104D50009F6F00012CEC22F00401B9D21EB041D1AA
:104D600084B820D188BD8BD004019E6B4DA608D09D
:104D70005250020805E252500A0802E3400E9E6FAC
:104D8000000188BF37D0070E04019F6F010EA06F8E
:104D9000000139EC21F088A11CD052520DE050C026
:104DA000A0F4770E0401A16FA26FA46BA36BA66B96
:104DB000A56B00018FDC0CD050C0A0F4770E04016D
:104DC000A16FA26BA46BA36BA66BA56B000182DC29
:104DD00010D0525004019E119F6F50C0A0F4770E66
:104DE000A16F9FC4A2F4A46BA36BA66BA56B00017B
:104DF00071DC45D0515243E03CEC16F0070E040143
:104E00009F6FA06B000139EC21F088A125D0525290
:104E100012E050C0A0F451C0A1F4770E0401A26FBB
:104E200059C0A4F458C0A3F45BC0A6F45AC0A5F4BA
:104E3000000150DC10D050C0A0F451C0A1F4040116
:104E4000A26B59C0A4F458C0A3F45BC0A6F45AC026
:104E5000A5F400013FDC13D0525004019E119F6F56
:104E600050C0A0F451C0A1F4A26F59C0A4F458C01E
:104E7000A3F45BC0A6F45AC0A5F400012BDC88B3F0
:104E800091D004019E6B4DA608D05650020805E251
:104E900056500A0802E3400E9E6F000188BF3AD0C8
:104EA000070E04019F6F010EA06F000139EC21F085
:104EB00088A11ED056520EE054C0A0F4770E040113
:104EC000A16FA26FA46BA36BA66BA56B00017DEC19
:104ED00022F00DD054C0A0F4770E0401A16FA26B94
:104EE000A46BA36BA66BA56B00017DEC22F011D027
:104EF000565004019E119F6F54C0A0F4770EA16F0D
:104F00009FC4A2F4A46BA36BA66BA56B00017DEC00
:104F100022F048D0555246E03CEC16F0070E040152
:104F20009F6FA06B000139EC21F088A127D0565269
:104F300013E054C0A0F455C0A1F4770E0401A26F91
:104F400059C0A4F458C0A3F45BC0A6F45AC0A5F499
:104F500000017DEC22F011D054C0A0F455C0A1F4A2
:104F60000401A26B59C0A4F458C0A3F45BC0A6F41A
:104F70005AC0A5F400017DEC22F014D05650040173
:104F80009E119F6F54C0A0F455C0A1F4A26F59C0E8
:104F9000A4F458C0A3F45BC0A6F45AC0A5F4000161
:104FA0007DEC22F00401835107081CE1040EEA6E37
:104FB000880EE96EF2CF9FF4F29E000E000137ECEE
:104FC00007F00A000900F550EE6E0009FBE104014C
:104FD0009FBFF28E040EA06F880E9F6F00012CEC15
:104FE00022F0040174D11EB06FD184B84ED188BDB7
:104FF000A5D004019E6B4DA608D05250020805E2D0
:1050000052500A0802E3400E9E6F000188B147D05B
:10501000090E04019F6F010EA06F000139EC21F011
:1050200088AF1ED051520EE050C0A0F4770E04019C
:10503000A16FA26FA46BA36BA66BA56B00016AECBA
:1050400023F00DD050C0A0F40401A16B770EA26F25
:10505000A46BA36BA66BA56B00016AEC23F01ED0BA
:105060003CEC16F0515208E059C085F458C084F465
:105070005BC087F45AC086F450C0A0F451C0A1F4BC
:10508000770E0401A26F85C4A4F484C4A3F487C47A
:10509000A6F486C4A5F400016AEC23F04FD0525266
:1050A0004DE0090E04019F6FA06B000139EC21F067
:1050B00088AF24D0515212E0525004019E119F6FCC
:1050C00050C0A0F4770EA16F9FC4A2F4A46BA36B91
:1050D000A66BA56B00016AEC23F00FD052500401BF
:1050E0009E119F6F50C0A0F4A16BA26FA46BA36B25
:1050F000A66BA56B00016AEC23F020D03CEC16F007
:10510000515208E059C085F458C084F45BC087F45C
:105110005AC086F4525004019E119F6F50C0A0F4F3
:1051200051C0A1F4A26F85C4A4F484C4A3F487C4BD
:10513000A6F486C4A5F400016AEC23F088B3A5D0D8
:1051400004019E6B4DA608D05650020805E2565049
:105150000A0802E3400E9E6F000188B147D0090E95
:1051600004019F6F010EA06F000139EC21F088AFA0
:105170001ED055520EE054C0A0F4770E0401A16F6A
:10518000A26FA46BA36BA66BA56B00017DEC22F054
:105190000DD054C0A0F40401A16B770EA26FA46BD4
:1051A000A36BA66BA56B00017DEC22F01ED03CEC3E
:1051B00016F0555208E059C085F458C084F45BC01D
:1051C00087F45AC086F454C0A0F455C0A1F4770EF9
:1051D0000401A26F85C4A4F484C4A3F487C4A6F414
:1051E00086C4A5F400017DEC22F04FD056524DE06C
:1051F000090E04019F6FA06B000139EC21F088AF0C
:1052000024D0555212E0565004019E119F6F54C095
:10521000A0F4770EA16F9FC4A2F4A46BA36BA66B3E
:10522000A56B00017DEC22F00FD0565004019E11B9
:105230009F6F54C0A0F4A16BA26FA46BA36BA66B6D
:10524000A56B00017DEC22F020D03CEC16F055520D
:1052500008E059C085F458C084F45BC087F45AC094
:1052600086F4565004019E119F6F54C0A0F455C09F
:10527000A1F4A26F85C4A4F484C4A3F487C4A6F4E3
:1052800086C4A5F400017DEC22F0040183510908D5
:105290001CE1040EEA6E880EE96EF2CF9FF4F29ED6
:1052A000000E00014FEC07F00A000900F550EE6E09
:1052B0000009FBE104019FBFF28E040EA06F880E6F
:1052C0009F6F00012CEC22F0040101D004010001C9
:1052D00046EF4CF0F2CF0DF0F29EE824F76AF73675
:1052E000FF0FF66E520EF722000EF86EFB6E0A00EC
:1052F000F550FA6E0800F5500DBEF28EF96E484971
:105300004849384A384AC84BC84B5C4D5C4DE64F5B
:10531000E64F0401BD6BBC6BBE6B300EBF6FC06F40
:10532000C16BC26BC36BC46B010EC56FC66BB9C4D6
:1053300003F0B851B9AF08D0000ED880B855006E50
:10534000000EB955036E0050BC6F03C0BDF4BC53D2
:1053500002E1BD5348E0BC5302E1BD532CE0036AB7
:10536000C551BE0FE96E040E0320EA6EBDC413F6EC
:10537000BCC412F60601156B0A0E146F000199ECFD
:1053800016F000C0C9F4040103C0CAF4005030098B
:10539000EF6EC52BBDC413F6BCC412F60601156B27
:1053A0000A0E146F000199EC16F002C0BDF401C0A2
:1053B000BCF40401D0D7B9BF01D00AD0036AC551EB
:1053C000BE0FE96E040E0320EA6E2D0EEF6EC52BA4
:1053D000036AC551BE0FE96E040E0320EA6EEF5258
:1053E00001E0C52B02D0030EC56FC5531BE0036A55
:1053F000C651BA25016EBB51032203C0C8F4010E89
:10540000C55D036ABE0FE96E040E0320EA6EEFCF9E
:10541000C9F4C8C4EAFF01C0E9FFC9C4EFFFC62B45
:10542000C507E3D700013CEF2AF00401B66B090E73
:10543000B76F040EEA6E890EE96E06010F6B116BF1
:10544000130E106F000187EC0FF0040EEA6E9C0E35
:10545000E96E06010F6B116B130E106F000187ECE4
:105460000FF088C4B9F487C4B8F4040E0401BB6F0C
:10547000AF0EBA6F00014DD7040E0601106FAF0ECC
:105480000F6F000125EC12F001C0B6F4036A0201AF
:10549000AD51B30FE96E020E0320EA6EEF50120D0C
:1054A000F350036A2F0F016E020E032201C0B8F4FD
:1054B000040103C0B9F4040EC86F890EC76F03C09E
:1054C000CAF401C0C9F4120ECB6F000178EC1AF0D7
:1054D0000C0E0401896F040EC86F890EC76F00019E
:1054E00083EC12F0050E0401CC6F0001B9EC0FF053
:1054F000DDBB25D088C400F887C4FFF70801026B24
:10550000120E016F00016BEC1CF002C003F00150A1
:10551000C20F016E020E032201C0B8F4040103C0E1
:10552000B9F4040EC86F9C0EC76F03C0CAF401C063
:10553000C9F4120ECB6F000178EC1AF066D0DDBD15
:105540002ED0040EEA6E9C0EE96E200E06010F6F3F
:10555000116B090E106F000187EC0FF00401B653B8
:105560001BE0036AB7519C0F016E040E032203C0B7
:10557000B9F4010EB65D036AAF0FE96E040E0320A5
:10558000EA6EEFCFBAF4B9C4EAFF01C0E9FFBAC4CA
:10559000EFFFB707B607E3D7A66B37D00001040EBD
:1055A000EA6E9C0EE96E200E06010F6F116B090E5C
:1055B000106F000187EC0FF00401B6531BE0036A83
:1055C000B7519C0F016E040E032203C0B9F4010E03
:1055D000B65D036AAF0FE96E040E0320EA6EEFCFEB
:1055E000BAF4B9C4EAFF01C0E9FFBAC4EFFFB707D4
:1055F000B607E3D7730EA76F650EA86F630EA96F8A
:10560000AA6BA5C4A6F42E0EA56F0A0E04019C6F0A
:105610003E0E9D6F040EC86F9C0EC76F000183EC99
:1056200012F0000CDD8F0201B751010A000103E006
:10563000030A10E01ED0030E0401876F3DC489F4F5
:105640003CC488F45BC08BF45AC08AF4000154EC6B
:105650001DF010D0020E0401876F59C089F458C0A4
:1056600088F43DC48BF43CC48AF4000154EC1DF072
:1056700001D000D0000C04013E513C5D09E13F51D6
:105680003D5D06E1010E405D3C6F000E41593D6FEE
:105690003C2BD8B43D2B3DC488F43CC487F40001B6
:1056A000C4DE0201AD51040803E10001BBDF0201C9
:1056B00000016AEF2BF0040EEA6E840EE96E06011B
:1056C0000F6B116B030E106F000187EC0FF0DDA95B
:1056D00002D0D1D771D1036A0201AD51AE0FE96E8C
:1056E000020E0320EA6EEF500208D8A495D0036A98
:1056F000AD51B30FE96E020E0320EA6EEF52D8B43B
:105700008BD0036AAD51B30FE96E020E0320EA6E2F
:10571000EF06AD534BE0036AAD51B30FE96E020ED5
:105720000320EA6EEF5242E1036AAD51AE0FE96E1B
:10573000020E0320EA6E020EEF6E036AAD51B80F3F
:10574000E96E020E0320EA6E010EEF5C0401876F22
:10575000036A0201AD51B80FE96E020E0320EA6E32
:10576000EFCF88F487C49AF488C49BF40001B7ECA7
:105770001AF0036A0201AD51B30F016E020E03224B
:10578000040103C088F4036A0201AD51B80FE96E49
:10579000020E0320EA6EEFCF89F4040188C4EAFF09
:1057A00001C0E9FF89C4EFFF35D00201036AAD51A2
:1057B000B30FE96E020E0320EA6EEF5216E1036AA0
:1057C000AD51B30FE96E020E0320EA6EEF2A036AB1
:1057D000AD51AE0FE96E020E0320EA6EEF6A010EC4
:1057E0000401846F856B0ED00201036AAD51AE0FC8
:1057F000E96E020E0320EA6E010EEF6E020E040146
:10580000846F856B040EC86F840EC76F000183EC34
:1058100012F00401D1D00201036AAD51B30FE96E59
:10582000020E0320EA6EEFCF87F4036AAD51BD0F7D
:10583000E96E020E0320EA6EEF500401875DD8B4D2
:105840007AD0D8A078D0036A0201AD51B30FE96EC7
:10585000020E0320EA6EEF06036AAD51B30FE96E44
:10586000020E0320EA6EEF50010849E3036AAD51CE
:10587000B30FE96E020E0320EA6EEF06AD5311E19D
:10588000036AAD51AE0FE96E020E0320EA6EEF6AB5
:10589000036AAD51B30FE96E020E0320EA6EEF6AA0
:1058A00012D0036AAD51B30FE96E020E0320EA6E07
:1058B000010EEF6E036AAD51AE0FE96E020E0320CA
:1058C000EA6E020EEF6E036AAD51BD0FE96E020E75
:1058D0000320EA6EEFCF87F4036AAD51BD0FE96E86
:1058E000020E0320EA6E010EEF240401886F87C4C4
:1058F0009AF49B6F0001B7EC1AF01BD00201036A07
:10590000AD51B30FE96E020E0320EA6EEFCF87F4BC
:10591000036AAD51B30FE96E020E0320EA6E010E69
:10592000EF240401886F87C49AF49B6F0001B7ECE1
:105930001AF042D00401036A0201AD51AE0FE96EC4
:10594000020E0320EA6E020EEF6E036AAD51B80F2D
:10595000E96E020E0320EA6E010EEF5C0401876F10
:10596000036A0201AD51B80FE96E020E0320EA6E20
:10597000EFCF88F487C49AF488C49BF40001B7EC95
:105980001AF0036A0201AD51B30F016E020E032239
:10599000040103C088F4036A0201AD51B80FE96E37
:1059A000020E0320EA6EEFCF89F4040188C4EAFFF7
:1059B00001C0E9FF89C4EFFF040196EF3CF0040148
:1059C00040513C5D09E141513D5D06E1010E3E253E
:1059D0003C6F000E3F213D6F3C51D8B43D073C0762
:1059E0003DC488F43CC487F400011FDD0201AD51C1
:1059F000040803E1000116DE020100010FEF2DF0A3
:105A0000040EEA6E840EE96E06010F6B116B030E35
:105A1000106F000187EC0FF0DDA902D0D0D7FFD0C6
:105A2000036A0201AD51AE0FE96E020E0320EA6E69
:105A3000EF50000A000105E0010A31E0030A4DE0E1
:105A4000EED0036A0201AD51B30FE96E020E0320DE
:105A5000EA6E020EEF6E036AAD51AE0FE96E020EF2
:105A60000320EA6E010EEF6E036AAD51B30FE96ECB
:105A7000020E0320EA6EEFCF87F4036AAD51B30F35
:105A8000E96E020E0320EA6E010EEF240401886F16
:105A900087C49AF49B6F0001B7EC1AF0C0D0036A78
:105AA0000201AD51B30FE96E020E0320EA6EEF2A38
:105AB000036AAD51AE0FE96E020E0320EA6E020ECC
:105AC000EF6E030E0401846F856B040EC86F840EA5
:105AD000C76F000183EC12F0A2D0036A0201AD513E
:105AE000B30FE96E020E0320EA6EEF2A036AAD518E
:105AF000B30FE96E020E0320EA6EEFCF87F4036A5C
:105B0000AD51B80FE96E020E0320EA6EEF500401AA
:105B1000875D67E066E30201AD5324E1036AAD519E
:105B2000AE0FE96E020E0320EA6EEF6A036AAD5112
:105B3000B30F016E020E0322040103C088F4036A4E
:105B40000201AD51BD0FE96E020E0320EA6EEFCFE8
:105B500089F4040188C4EAFF01C0E9FF89C4EFFFAA
:105B600023D00201036AAD51AE0FE96E020E03208D
:105B7000EA6E020EEF6E036AAD51B30F016E020EB4
:105B80000322040103C088F4036A0201AD51BD0F72
:105B9000E96E020E0320EA6E010EEF24040188C4B0
:105BA000EAFF01C0E9FFEF6E036A0201AD51BD0FCC
:105BB000E96E020E0320EA6EEFCF87F4036AAD515F
:105BC000BD0FE96E020E0320EA6E010EEF24040100
:105BD000886F87C49AF49B6F0001B7EC1AF01ED04F
:105BE0000401036A0201AD51B30FE96E020E0320F6
:105BF000EA6E010EEF5C0401876F036A0201AD518A
:105C0000B30FE96E020E0320EA6EEFCF88F487C46B
:105C10009AF488C49BF40001B7EC1AF000D08CEF22
:105C20003CF0C8EF32F0AA6AA96A4DC0A8FFA69C52
:105C3000A69EA684F250006EF29E0F01550EA76E2E
:105C4000AA0EA76EA682A6B2FED7A6940050F212A4
:105C5000AA6A010EA96E4EC0A8FFA69CA69EA684A5
:105C6000F2CF00F0F29E550EA76EAA0EA76EA68286
:105C7000A6B2FED7A6940050F212AA6A020EA96E2E
:105C800050C0A8FFA69CA69EA684F2CF00F0F29E6C
:105C9000550EA76EAA0EA76EA682A6B2FED7A69430
:105CA0000050F212AA6A030EA96E51C0A8FFA69C6A
:105CB000A69EA684F2CF00F0F29E550EA76EAA0E05
:105CC000A76EA682A6B2FED7A6940050F212AA6AC8
:105CD000040EA96E52C0A8FFA69CA69EA684F2CF71
:105CE00000F0F29E550EA76EAA0EA76EA682A6B26F
:105CF000FED7A6940050F212AA6A050EA96E54C0EF
:105D0000A8FFA69CA69EA684F2CF00F0F29E550E98
:105D1000A76EAA0EA76EA682A6B2FED7A6940050C2
:105D2000F212AA6A060EA96E55C0A8FFA69CA69EEE
:105D3000A684F2CF00F0F29E550EA76EAA0EA76EB3
:105D4000A682A6B2FED7A6940050F212AA6A070E47
:105D5000A96E56C0A8FFA69CA69EA684F2CF00F00E
:105D6000F29E550EA76EAA0EA76EA682A6B2FED709
:105D7000A6940050F2120001000C010E0201B45D65
:105D8000FB0FD8B08DD0050F000153EF2FF0000EA0
:105D90004DB2010E036A04013C5D1CE103503D5D00
:105DA00019E13C530BE13D5309E14D82160E06010A
:105DB0000F6F0001BCEC16F00CD004013C2D0AD092
:105DC0003D5308E14D92170E06010F6F0001BCEC28
:105DD00016F00401000127DF020162D004013C53E8
:105DE00004E13D5302E14D8405D03C2D03D03D53E9
:105DF00001E14D94000117DF020152D004013C5330
:105E000008E13D5306E1130E06010F6F0001BCECE3
:105E100016F0020145D0000E4DB6010E036A0401D2
:105E20003C5D0CE103503D5D09E13C5304E13D5311
:105E300002E14D8601D04D960001F5DE020130D021
:105E400004013C530FE13D530DE11EB00AD01E800A
:105E50001E921D0E06010F6F0001BCEC16F0E3DE72
:105E600004011BD03C2D10D03D530EE11EA00BD0E1
:105E70001EB209D01E821D0E06010F6F0001BCEC80
:105E800016F0D1DE040109D01E901E921E0E0601EE
:105E90000F6F0001BCEC16F0C6DE020101D002015A
:105EA0000201D7EF32F0F2CF0DF0F29EE824F76A4C
:105EB000F736D10FF66E5E0EF722000EF86EFB6E0F
:105EC0000A00F550FA6E0800F5500DBEF28EF96E1C
:105ED0008E5DDC5DFC5D165E405E0401882D09D0A0
:105EE000505206E0515201E0556A525201E0566AA2
:105EF00008D0545206E0555201E0516A565201E072
:105F0000526A0001000C0401856B846B876B866B01
:105F10000201B551010A000106E0030A5BE0010A33
:105F2000D8B4AFD005D1036A505004013C5D03E101
:105F300003503D5D4DE03CC450F000013CEC16F0D8
:105F4000515208E059C085F458C084F45BC087F40E
:105F50005AC086F450C0A0F451C0A1F452C0A2F4BB
:105F600085C4A4F484C4A3F487C4A6F486C4A5F4A9
:105F70006AEC23F0010E0401886F0001AEDF04011A
:105F8000856B846B876B866B00013CEC16F0555279
:105F900008E059C085F458C084F45BC087F45AC047
:105FA00086F454C0A0F455C0A1F456C0A2F485C430
:105FB000A4F484C4A3F487C4A6F486C4A5F47DEC39
:105FC00022F031DE040E06010F6F0001BCEC16F06A
:105FD0000001AED0036A515004013C5D03E103505F
:105FE0003D5D4DE03CC451F000013CEC16F05152D7
:105FF00008E059C085F458C084F45BC087F45AC0E7
:1060000086F450C0A0F451C0A1F452C0A2F485C4DB
:10601000A4F484C4A3F487C4A6F486C4A5F46AECEB
:1060200023F0010E0401886F000157DF0401856B26
:10603000846B876B866B00013CEC16F0555208E0D0
:1060400059C085F458C084F45BC087F45AC086F404
:1060500054C0A0F455C0A1F456C0A2F485C4A4F461
:1060600084C4A3F487C4A6F486C4A5F47DEC22F00E
:10607000DADD040E06010F6F0001BCEC16F0000122
:1060800057D0036A525004013C5D03E103503D5D6B
:106090004DE03CC452F000013CEC16F0515208E0D7
:1060A00059C085F458C084F45BC087F45AC086F4A4
:1060B00050C0A0F451C0A1F452C0A2F485C4A4F40D
:1060C00084C4A3F487C4A6F486C4A5F46AEC23F0C0
:1060D000010E0401886F000100DF0401856B846BF1
:1060E000876B866B00013CEC16F0555208E059C0F6
:1060F00085F458C084F45BC087F45AC086F454C059
:10610000A0F455C0A1F456C0A2F485C4A4F484C47C
:10611000A3F487C4A6F486C4A5F47DEC22F083DD45
:10612000040E06010F6F0001BCEC16F0000100D058
:10613000CFEF32F00401856B846B876B866B0201B5
:10614000B651010A000106E0030A5AE0010AD8B478
:10615000ADD002D1036A545004013C5D03E1035009
:106160003D5D4CE03CC454F000013CEC16F055524F
:1061700008E059C085F458C084F45BC087F45AC065
:1061800086F454C0A0F455C0A1F456C0A2F485C44E
:10619000A4F484C4A3F487C4A6F486C4A5F47DEC57
:1061A00022F00401886B000198DE0401856B846B8A
:1061B000876B866B00013CEC16F0515208E059C029
:1061C00085F458C084F45BC087F45AC086F450C08C
:1061D000A0F451C0A1F452C0A2F485C4A4F484C4B4
:1061E000A3F487C4A6F486C4A5F46AEC23F01BDDEF
:1061F000060E06010F6F0001BCEC16F00001ACD0DA
:10620000036A555004013C5D03E103503D5D4CE0E1
:106210003CC455F000013CEC16F0555208E059C062
:1062200085F458C084F45BC087F45AC086F454C027
:10623000A0F455C0A1F456C0A2F485C4A4F484C44B
:10624000A3F487C4A6F486C4A5F47DEC22F004016F
:10625000886B000142DE0401856B846B876B866B63
:1062600000013CEC16F0515208E059C085F458C0CA
:1062700084F45BC087F45AC086F450C0A0F451C0C7
:10628000A1F452C0A2F485C4A4F484C4A3F487C4C6
:10629000A6F486C4A5F46AEC23F0C5DC060E06015C
:1062A0000F6F0001BCEC16F0000156D0036A565087
:1062B00004013C5D03E103503D5D4CE03CC456F0FD
:1062C00000013CEC16F0555208E059C085F458C066
:1062D00084F45BC087F45AC086F454C0A0F455C05F
:1062E000A1F456C0A2F485C4A4F484C4A3F487C462
:1062F000A6F486C4A5F47DEC22F00401886B0001AD
:10630000ECDD0401856B846B876B866B00013CECD4
:1063100016F0515208E059C085F458C084F45BC0AF
:1063200087F45AC086F450C0A0F451C0A1F452C002
:10633000A2F485C4A4F484C4A3F487C4A6F486C4D8
:10634000A5F46AEC23F06FDC060E06010F6F000166
:10635000BCEC16F0000100D0D2EF32F00401856BE6
:10636000846B876B515006081AE25150110817E3ED
:10637000070E515C006ED89000360050036A5C0F27
:10638000E96E000E0320EA6E59C0ECFFED5258C0D2
:10639000EFFF070E515C006ED8900034876F5550A8
:1063A00006081AE25550110817E3070E555C006EF7
:1063B000D89000360050036A5C0FE96E000E03208F
:1063C000EA6E59C0ECFFED5258C0EFFF070E555C66
:1063D000006ED8900034876F100E8725846F856B10
:1063E00059C086F485C4AAFF84C4A9FF86C4A8FF47
:1063F000A69CA69EA684F250006EF29E0F01550E3A
:10640000A76EAA0EA76EA682A6B2FED7A6940050CB
:10641000F212010E04018427000E852358C086F471
:1064200085C4AAFF84C4A9FF86C4A8FFA69CA69E13
:10643000A684F250006EF29E0F01550EA76EAA0EB2
:10644000A76EA682A6B2FED7A6940050F212000153
:10645000BCEF32F00401856B846B876B51500608EA
:106460001AE25150110817E3070E515C006ED890E4
:1064700000360050036A720FE96E000E0320EA6EC8
:106480005BC0ECFFED525AC0EFFF070E515C006E8F
:10649000D8900034876F555006081AE255501108FD
:1064A00017E3070E555C006ED89000360050036A63
:1064B000720FE96E000E0320EA6E5BC0ECFFED5236
:1064C0005AC0EFFF070E555C006ED8900034876FFE
:1064D000260E8725846F856B5BC086F485C4AAFF72
:1064E00084C4A9FF86C4A8FFA69CA69EA684F250D9
:1064F000006EF29E0F01550EA76EAA0EA76EA68221
:10650000A6B2FED7A6940050F212010E0401842711
:10651000000E85235AC086F485C4AAFF84C4A9FF4F
:1065200086C4A8FFA69CA69EA684F250006EF29E8A
:106530000F01550EA76EAA0EA76EA682A6B2FED7B1
:10654000A6940050F2120001BCEF32F0DD9F020170
:10655000B751010A000103E0030A07E00CD03DC473
:1065600059F03CC458F0FAD607D03DC45BF03CC4A7
:106570005AF070D701D000D0D5EF32F00201AD5102
:10658000FB0F15E2050F0001DCEF32F011EF2EF0EA
:1065900002010DD0BDEF2EF0020109D0B4D40201EA
:1065A00006D0C8D5020103D0D1D7020100D0000126
:1065B000F5EC1DF052EF3CF0F2CF0DF0F29EE82426
:1065C000F76AF736E30FF66E650EF722000EF86EE7
:1065D000FB6E0A00F550FA6E0800F5500DBEF28E03
:1065E000F96E8C6594659C65A265A8650201B3513E
:1065F000020A000107E0010A22E0060A3DE0010A62
:1066000058E074D0020E0401996F0001D5EC17F028
:10661000036A0201AD51B30FE96E020E0320EA6E68
:10662000010EEF6E036AAD51AE0FE96E020E03204C
:10663000EA6E020EEF6E000120EC1EF05BD0030E3E
:106640000401996F0001D5EC17F0036A0201AD5106
:10665000B30FE96E020E0320EA6E010EEF6E036ABD
:10666000AD51AE0FE96E020E0320EA6E020EEF6E20
:10667000000120EC1EF03ED0010E0401996F0001D4
:10668000D5EC17F0036A0201AD51B30FE96E020EAB
:106690000320EA6E010EEF6E036AAD51AE0FE96E94
:1066A000020E0320EA6E020EEF6E000120EC1EF0D7
:1066B00021D0040E0401996F0001D5EC17F0036A94
:1066C0000201AD51B30FE96E020E0320EA6E010E16
:1066D000EF6E036AAD51AE0FE96E020E0320EA6E53
:1066E000020EEF6E000120EC1EF004D0DD99DD9B60
:1066F000DD9D00D073EF3CF00201B451030A0001AC
:106700000BE0020A25E0030A23E0060AD8B46ED0A3
:10671000010AD8B49DD0EAD0020EEA6EC20EE96E2C
:10672000F2CF84F4F29E000EA8EC09F00A000900F2
:10673000F550EE6E0009FBE1040184BFF28E3F6B61
:106740003E6B3D6B3C6B3DC441F43CC440F4D3D044
:10675000020EEA6EC20EE96EF2CF84F4F29E000ED3
:10676000BDEC09F00A000900F550EE6E0009FBE1EE
:10677000040184BFF28E020EEA6ED40EE96EF2CFEF
:1067800084F4F29E000E0001D2EC09F00A00090028
:10679000F550EE6E0009FBE1040184BFF28E036A3E
:1067A0000201AD51B30FE96E020E0320EA6EEF5005
:1067B000010A000103E0030A08E00ED0000E4DA21A
:1067C000010E04013D6B3C6F0BD0000E4DA4010E79
:1067D00004013D6B3C6F04D004013D6B3C6B00D069
:1067E0003F6B010E3E6F416B406B85D0020EEA6E2F
:1067F000C20EE96EF2CF84F4F29E000EE7EC09F0CF
:106800000A000900F550EE6E0009FBE1040184BFA7
:10681000F28E020EEA6ED40EE96EF2CF84F4F29E8E
:10682000000E0001FCEC09F00A000900F550EE6EC4
:106830000009FBE1040184BFF28E000E4DA6010E9B
:106840003D6B3C6F3F6B010E3E6F416B406B53D015
:10685000020EEA6EC20EE96EF2CF84F4F29E000ED2
:1068600011EC0AF00A000900F550EE6E0009FBE198
:10687000040184BFF28E020EEA6ED40EE96EF2CFEE
:1068800084F4F29E000E000125EC0AF00A000900D3
:10689000F550EE6E0009FBE1040184BFF28E020E9A
:1068A000EA6EE60EE96EF2CF84F4F29E000E00016D
:1068B000FCEC09F00A000900F550EE6E0009FBE15E
:1068C000040184BFF28E3D6B020E3C6F1EA007D008
:1068D0003D6B3C6B1EA203D03D6B010E3C6F416BC8
:1068E000406B3F6B020E3E6F06D00001DD99DD9BD1
:1068F000DD9D040100D0000173EF3CF0DD9BDD9DC8
:106900000201B551010A000108E0030AD8B4B1D16F
:10691000010AD8B446D3B6EF38F0020EEA6EC20EC2
:10692000E96EF2CF84F4F29E000E39EC0AF00A0010
:106930000900F550EE6E0009FBE1040184BFF28E00
:10694000020EEA6ED40EE96EF2CF84F4F29E000ECF
:10695000000151EC0AF00A000900F550EE6E000942
:10696000FBE1040184BFF28E020EEA6EE60EE96ED0
:10697000F2CF84F4F29E000E000169EC0AF00A00E6
:106980000900F550EE6E0009FBE1040184BFF28EB0
:10699000020EEA6EF80EE96EF2CF84F4F29E000E5B
:1069A000000181EC0AF00A000900F550EE6E0009C2
:1069B000FBE1040184BFF28E030EEA6E0A0EE96E5B
:1069C000F2CF84F4F29E000E000199EC0AF00A0066
:1069D0000900F550EE6E0009FBE1040184BFF28E60
:1069E000030EEA6E1C0EE96EF2CF84F4F29E000EE6
:1069F0000001B1EC0AF00A000900F550EE6E000942
:106A0000FBE1040184BFF28E030EEA6E2E0EE96EE6
:106A1000F2CF84F4F29E000E0001C9EC0AF00A00E5
:106A20000900F550EE6E0009FBE1040184BFF28E0F
:106A3000030EEA6E400EE96EF2CF84F4F29E000E71
:106A40000001E1EC0AF00A000900F550EE6E0009C1
:106A5000FBE1040184BFF28E030EEA6E520EE96E72
:106A6000F2CF84F4F29E000E0001F9EC0AF00A0065
:106A70000900F550EE6E0009FBE1040184BFF28EBF
:106A8000030EEA6E640EE96EF2CF84F4F29E000EFD
:106A9000000111EC0BF00A000900F550EE6E000940
:106AA000FBE1040184BFF28E030EEA6E760EE96EFE
:106AB000F2CF84F4F29E000E000129EC0BF00A00E4
:106AC0000900F550EE6E0009FBE1040184BFF28E6F
:106AD000030EEA6E880EE96EF2CF84F4F29E000E89
:106AE000000141EC0BF00A000900F550EE6E0009C0
:106AF000FBE1040184BFF28E030EEA6E9A0EE96E8A
:106B0000F2CF84F4F29E000E000159EC0BF00A0063
:106B10000900F550EE6E0009FBE1040184BFF28E1E
:106B2000030EEA6EAC0EE96EF2CF84F4F29E000E14
:106B3000000171EC0BF00A000900F550EE6E00093F
:106B4000FBE1040184BFF28E030EEA6EBE0EE96E15
:106B5000F2CF84F4F29E000E000189EC0BF00A00E3
:106B60000900F550EE6E0009FBE1040184BFF28ECE
:106B7000030EEA6ED00EE96EF2CF84F4F29E000EA0
:106B80000001A1EC0BF00A000900F550EE6E0009BF
:106B9000FBE1040184BFF28E030EEA6EE20EE96EA1
:106BA000F2CF84F4F29E000E0001B9EC0BF00A0063
:106BB0000900F550EE6E0009FBE1040184BFF28E7E
:106BC000030EEA6EF40EE96EF2CF84F4F29E000E2C
:106BD0000001D1EC0BF00A000900F550EE6E00093F
:106BE000FBE1040184BFF28E040EEA6E060EE96E2C
:106BF000F2CF84F4F29E000E0001E9EC0BF00A00E3
:106C00000900F550EE6E0009FBE1040184BFF28E2D
:106C1000040EEA6E180EE96EF2CF84F4F29E000EB6
:106C2000000101EC0CF00A000900F550EE6E0009BD
:106C3000FBE1040184BFF28E040EEA6E2A0EE96EB7
:106C4000F2CF84F4F29E000E000119EC0CF00A0061
:106C50000900F550EE6E0009FBE1040184BFF28EDD
:106C60003F6B140E3E6F416B406B3D6B50C03CF46C
:106C700080D2020EEA6EC20EE96EF2CF84F4F29E6A
:106C8000000E31EC0CF00A000900F550EE6E000920
:106C9000FBE1040184BFF28E020EEA6ED40EE96EAF
:106CA000F2CF84F4F29E000E000151EC0AF00A00CB
:106CB0000900F550EE6E0009FBE1040184BFF28E7D
:106CC000020EEA6EE60EE96EF2CF84F4F29E000E3A
:106CD000000169EC0AF00A000900F550EE6E0009A7
:106CE000FBE1040184BFF28E020EEA6EF80EE96E3B
:106CF000F2CF84F4F29E000E000181EC0AF00A004B
:106D00000900F550EE6E0009FBE1040184BFF28E2C
:106D1000030EEA6E0A0EE96EF2CF84F4F29E000EC4
:106D2000000199EC0AF00A000900F550EE6E000926
:106D3000FBE1040184BFF28E030EEA6E1C0EE96EC5
:106D4000F2CF84F4F29E000E0001B1EC0AF00A00CA
:106D50000900F550EE6E0009FBE1040184BFF28EDC
:106D6000030EEA6E2E0EE96EF2CF84F4F29E000E50
:106D70000001C9EC0AF00A000900F550EE6E0009A6
:106D8000FBE1040184BFF28E030EEA6E400EE96E51
:106D9000F2CF84F4F29E000E000149EC0CF00A00E0
:106DA0000900F550EE6E0009FBE1040184BFF28E8C
:106DB000030EEA6E520EE96EF2CF84F4F29E000EDC
:106DC0000001E1EC0AF00A000900F550EE6E00093E
:106DD000FBE1040184BFF28E030EEA6E640EE96EDD
:106DE000F2CF84F4F29E000E0001F9EC0AF00A00E2
:106DF0000900F550EE6E0009FBE1040184BFF28E3C
:106E0000030EEA6E760EE96EF2CF84F4F29E000E67
:106E1000000111EC0BF00A000900F550EE6E0009BC
:106E2000FBE1040184BFF28E030EEA6E880EE96E68
:106E3000F2CF84F4F29E000E000129EC0BF00A0060
:106E40000900F550EE6E0009FBE1040184BFF28EEB
:106E5000030EEA6E9A0EE96EF2CF84F4F29E000EF3
:106E6000000141EC0BF00A000900F550EE6E00093C
:106E7000FBE1040184BFF28E030EEA6EAC0EE96EF4
:106E8000F2CF84F4F29E000E000159EC0BF00A00E0
:106E90000900F550EE6E0009FBE1040184BFF28E9B
:106EA000030EEA6EBE0EE96EF2CF84F4F29E000E7F
:106EB000000171EC0BF00A000900F550EE6E0009BC
:106EC000FBE1040184BFF28E030EEA6ED00EE96E80
:106ED000F2CF84F4F29E000E000189EC0BF00A0060
:106EE0000900F550EE6E0009FBE1040184BFF28E4B
:106EF000030EEA6EE20EE96EF2CF84F4F29E000E0B
:106F00000001A1EC0BF00A000900F550EE6E00093B
:106F1000FBE1040184BFF28E030EEA6EF40EE96E0B
:106F2000F2CF84F4F29E000E0001B9EC0BF00A00DF
:106F30000900F550EE6E0009FBE1040184BFF28EFA
:106F4000040EEA6E060EE96EF2CF84F4F29E000E95
:106F5000000161EC0CF00A000900F550EE6E00092A
:106F6000FBE1040184BFF28E040EEA6E180EE96E96
:106F7000F2CF84F4F29E000E000179EC0CF00A00CE
:106F80000900F550EE6E0009FBE1040184BFF28EAA
:106F90003F6B130E3E6F416B406B3D6B51C03CF439
:106FA000E8D0020EEA6EC20EE96EF2CF84F4F29ED1
:106FB000000E31EC0CF00A000900F550EE6E0009ED
:106FC000FBE1040184BFF28E020EEA6ED40EE96E7C
:106FD000F2CF84F4F29E000E000151EC0AF00A0098
:106FE0000900F550EE6E0009FBE1040184BFF28E4A
:106FF000020EEA6EE60EE96EF2CF84F4F29E000E07
:10700000000169EC0AF00A000900F550EE6E000973
:10701000FBE1040184BFF28E020EEA6EF80EE96E07
:10702000F2CF84F4F29E000E000190EC0CF00A0006
:107030000900F550EE6E0009FBE1040184BFF28EF9
:10704000030EEA6E0A0EE96EF2CF84F4F29E000E91
:107050000001A8EC0CF00A000900F550EE6E0009E2
:10706000FBE1040184BFF28E030EEA6E1C0EE96E92
:10707000F2CF84F4F29E000E000181EC0AF00A00C7
:107080000900F550EE6E0009FBE1040184BFF28EA9
:10709000030EEA6E2E0EE96EF2CF84F4F29E000E1D
:1070A000000199EC0AF00A000900F550EE6E0009A3
:1070B000FBE1040184BFF28E030EEA6E400EE96E1E
:1070C000F2CF84F4F29E000E0001B1EC0AF00A0047
:1070D0000900F550EE6E0009FBE1040184BFF28E59
:1070E000030EEA6E520EE96EF2CF84F4F29E000EA9
:1070F0000001C9EC0AF00A000900F550EE6E000923
:10710000FBE1040184BFF28E030EEA6E640EE96EA9
:10711000F2CF84F4F29E000E0001C0EC0CF00A00E5
:107120000900F550EE6E0009FBE1040184BFF28E08
:10713000030EEA6E760EE96EF2CF84F4F29E000E34
:107140000001D8EC0CF00A000900F550EE6E0009C1
:10715000FBE1040184BFF28E3F6B0A0E3E6F416B70
:10716000406B3D6B52C03CF404D00001DD9904013A
:1071700000D0000173EF3CF0DD9BDD9D0201B651B4
:10718000010A000107E0030AD8B4E8D0010AD8B424
:107190007DD261D3020EEA6EC20EE96EF2CF84F4A4
:1071A000F29E000E39EC0AF00A000900F550EE6E6E
:1071B0000009FBE1040184BFF28E020EEA6ED40ED8
:1071C000E96EF2CF84F4F29E000E000151EC0AF059
:1071D0000A000900F550EE6E0009FBE1040184BFCE
:1071E000F28E020EEA6EE60EE96EF2CF84F4F29EA3
:1071F000000E000169EC0AF00A000900F550EE6E7D
:107200000009FBE1040184BFF28E020EEA6EF80E63
:10721000E96EF2CF84F4F29E000E000190EC0CF0C7
:107220000A000900F550EE6E0009FBE1040184BF7D
:10723000F28E030EEA6E0A0EE96EF2CF84F4F29E2D
:10724000000E0001A8EC0CF00A000900F550EE6EEB
:107250000009FBE1040184BFF28E030EEA6E1C0EEE
:10726000E96EF2CF84F4F29E000E000181EC0AF088
:107270000A000900F550EE6E0009FBE1040184BF2D
:10728000F28E030EEA6E2E0EE96EF2CF84F4F29EB9
:10729000000E000199EC0AF00A000900F550EE6EAC
:1072A0000009FBE1040184BFF28E030EEA6E400E7A
:1072B000E96EF2CF84F4F29E000E0001B1EC0AF008
:1072C0000A000900F550EE6E0009FBE1040184BFDD
:1072D000F28E030EEA6E520EE96EF2CF84F4F29E45
:1072E000000E0001C9EC0AF00A000900F550EE6E2C
:1072F0000009FBE1040184BFF28E030EEA6E640E06
:10730000E96EF2CF84F4F29E000E0001C0EC0CF0A6
:107310000A000900F550EE6E0009FBE1040184BF8C
:10732000F28E030EEA6E760EE96EF2CF84F4F29ED0
:10733000000E0001D8EC0CF00A000900F550EE6ECA
:107340000009FBE1040184BFF28E3F6B0A0E3E6F21
:10735000416B406B3D6B54C03CF480D2020EEA6E30
:10736000C20EE96EF2CF84F4F29E000E31EC0CF006
:107370000A000900F550EE6E0009FBE1040184BF2C
:10738000F28E020EEA6ED40EE96EF2CF84F4F29E13
:10739000000E000151EC0AF00A000900F550EE6EF3
:1073A0000009FBE1040184BFF28E020EEA6EE60ED4
:1073B000E96EF2CF84F4F29E000E000169EC0AF04F
:1073C0000A000900F550EE6E0009FBE1040184BFDC
:1073D000F28E020EEA6EF80EE96EF2CF84F4F29E9F
:1073E000000E000181EC0AF00A000900F550EE6E73
:1073F0000009FBE1040184BFF28E030EEA6E0A0E5F
:10740000E96EF2CF84F4F29E000E000199EC0AF0CE
:107410000A000900F550EE6E0009FBE1040184BF8B
:10742000F28E030EEA6E1C0EE96EF2CF84F4F29E29
:10743000000E0001B1EC0AF00A000900F550EE6EF2
:107440000009FBE1040184BFF28E030EEA6E2E0EEA
:10745000E96EF2CF84F4F29E000E0001C9EC0AF04E
:107460000A000900F550EE6E0009FBE1040184BF3B
:10747000F28E030EEA6E400EE96EF2CF84F4F29EB5
:10748000000E000149EC0CF00A000900F550EE6E08
:107490000009FBE1040184BFF28E030EEA6E520E76
:1074A000E96EF2CF84F4F29E000E0001E1EC0AF0E6
:1074B0000A000900F550EE6E0009FBE1040184BFEB
:1074C000F28E030EEA6E640EE96EF2CF84F4F29E41
:1074D000000E0001F9EC0AF00A000900F550EE6E0A
:1074E0000009FBE1040184BFF28E030EEA6E760E02
:1074F000E96EF2CF84F4F29E000E000111EC0BF065
:107500000A000900F550EE6E0009FBE1040184BF9A
:10751000F28E030EEA6E880EE96EF2CF84F4F29ECC
:10752000000E000129EC0BF00A000900F550EE6E88
:107530000009FBE1040184BFF28E030EEA6E9A0E8D
:10754000E96EF2CF84F4F29E000E000141EC0BF0E4
:107550000A000900F550EE6E0009FBE1040184BF4A
:10756000F28E030EEA6EAC0EE96EF2CF84F4F29E58
:10757000000E000159EC0BF00A000900F550EE6E08
:107580000009FBE1040184BFF28E030EEA6EBE0E19
:10759000E96EF2CF84F4F29E000E000171EC0BF064
:1075A0000A000900F550EE6E0009FBE1040184BFFA
:1075B000F28E030EEA6ED00EE96EF2CF84F4F29EE4
:1075C000000E000189EC0BF00A000900F550EE6E88
:1075D0000009FBE1040184BFF28E030EEA6EE20EA5
:1075E000E96EF2CF84F4F29E000E0001A1EC0BF0E4
:1075F0000A000900F550EE6E0009FBE1040184BFAA
:10760000F28E030EEA6EF40EE96EF2CF84F4F29E6F
:10761000000E0001B9EC0BF00A000900F550EE6E07
:107620000009FBE1040184BFF28E040EEA6E060E2F
:10763000E96EF2CF84F4F29E000E000161EC0CF0D2
:107640000A000900F550EE6E0009FBE1040184BF59
:10765000F28E040EEA6E180EE96EF2CF84F4F29EFA
:10766000000E000179EC0CF00A000900F550EE6EF6
:107670000009FBE1040184BFF28E3F6B130E3E6FE5
:10768000416B406B3D6B55C03CF4E8D0020EEA6E96
:10769000C20EE96EF2CF84F4F29E000E31EC0CF0D3
:1076A0000A000900F550EE6E0009FBE1040184BFF9
:1076B000F28E020EEA6ED40EE96EF2CF84F4F29EE0
:1076C000000E000151EC0AF00A000900F550EE6EC0
:1076D0000009FBE1040184BFF28E020EEA6EE60EA1
:1076E000E96EF2CF84F4F29E000E000169EC0AF01C
:1076F0000A000900F550EE6E0009FBE1040184BFA9
:10770000F28E020EEA6EF80EE96EF2CF84F4F29E6B
:10771000000E000190EC0CF00A000900F550EE6E2E
:107720000009FBE1040184BFF28E030EEA6E0A0E2B
:10773000E96EF2CF84F4F29E000E0001A8EC0CF08A
:107740000A000900F550EE6E0009FBE1040184BF58
:10775000F28E030EEA6E1C0EE96EF2CF84F4F29EF6
:10776000000E000181EC0AF00A000900F550EE6EEF
:107770000009FBE1040184BFF28E030EEA6E2E0EB7
:10778000E96EF2CF84F4F29E000E000199EC0AF04B
:107790000A000900F550EE6E0009FBE1040184BF08
:1077A000F28E030EEA6E400EE96EF2CF84F4F29E82
:1077B000000E0001B1EC0AF00A000900F550EE6E6F
:1077C0000009FBE1040184BFF28E030EEA6E520E43
:1077D000E96EF2CF84F4F29E000E0001C9EC0AF0CB
:1077E0000A000900F550EE6E0009FBE1040184BFB8
:1077F000F28E030EEA6E640EE96EF2CF84F4F29E0E
:10780000000E0001C0EC0CF00A000900F550EE6E0D
:107810000009FBE1040184BFF28E030EEA6E760ECE
:10782000E96EF2CF84F4F29E000E0001D8EC0CF069
:107830000A000900F550EE6E0009FBE1040184BF67
:10784000F28E3F6B0A0E3E6F416B406B3D6B56C034
:107850003CF404D00001DD99040100D0000173EF75
:107860003CF0DD8B04013F6BFF0E3E6F416F010E5C
:10787000406F0201B751010A000103E0030A06E06C
:107880000AD059C03DF458C03CF406D05BC03DF46A
:107890005AC03CF401D000D073EF3CF0DDA903D016
:1078A000BEEF32F028D0DD890201AD51000A00019F
:1078B0000BE0010A0CE0030A0DE0010A0EE0070AE2
:1078C0000EE0010A0EE00DD0F6EF32F00CD07CEFA6
:1078D00033F009D07EEF34F006D04ED404D0C1D7B7
:1078E00002D0DD9900D0DDA906D03DC488F43CC4A7
:1078F00087F415EC2AF08FEF3CF00B0E0401835D4A
:10790000FC0F14E2040F000199EF3CF05BEF2BF049
:1079100004010CD000EF2DF0040108D0BFD7040102
:1079200005D020EC1EF0040101D00401000158EF45
:107930004CF0F2CF0DF0F29EE824F76AF7365D0FB7
:10794000F66E790EF722000EF86EFB6E0A00F55007
:10795000FA6E0800F5500DBEF28EF96E0C791479AE
:107960001C792279EF5210E0EACF2BF5E9CF2AF506
:10797000EF509EA8FED7AD6E2BC5EAFF2AC5E9FFE2
:10798000E92AD8B4EA2AEED7000C0900F55211E032
:10799000F6CF00F8F7CF01F8F8CF02F8F5509EA81F
:1079A000FED7AD6E00C8F6FF01C8F7FF02C8F8FFAA
:1079B000ECD7000C0401986B996B2B0E9A6F2D0E6F
:1079C0009B6F9C6F9D6F9E6F9F6FA06FA16FA26F4B
:1079D000A36FA46FA56FA66FA76FA86FA96FAA6FFB
:1079E000AB6FAC6FAD6FAE6FAF6FB06FB16FB26FAB
:1079F000B36FB46FB56FB66FB76FB86FB96FBA6F5B
:107A0000BB6FBC6FBD6FBE6FBF6FC06FC16FC26F0A
:107A1000C36FC46FC56FC66FC76FC86FC96FCA6FBA
:107A2000CB6FCC6FCD6FCE6FCF6FD06FD16FD26F6A
:107A3000D36FD46FD56FD66FD76FD86FD96FDA6F1A
:107A4000DB6FDC6FDD6FDE6FDF6FE06FE16FE26FCA
:107A5000E36FE46FE56FE66F2B0EE76FE86B7C0E6C
:107A6000E96F200EEA6FEB6FEC6FED6FEE6FEF6F6B
:107A7000F06FF16FF26FF36FF46FF56FF66FF76FF2
:107A8000F86FF96FFA6FFB6FFC6FFD6FFE6FFF6FA2
:107A90000501006F016F026F560E036F610E046FD8
:107AA000640E056F066F690E076F6F0E086F200E6C
:107AB000096F550E0A6F580E0B6F480E0C6F440E6F
:107AC0000D6F200E0E6F430E0F6F720E106F6F0E44
:107AD000116F730E126F136F500E146F6F0E156FC0
:107AE000690E166F6E0E176F740E186F200E196FD9
:107AF0001A6F1B6F1C6F1D6F1E6F1F6F206F216F22
:107B0000226F236F246F256F266F276F286F296FD1
:107B10002A6F2B6F2C6F2D6F2E6F2F6F306F316F81
:107B2000326F336F346F356F7C0E366F376B2B0EC1
:107B3000386F2D0E396F3A6F3B6F3C6F3D6F3E6F64
:107B40003F6F406F416F426F436F446F456F466FA9
:107B5000476F486F496F4A6F4B6F4C6F4D6F4E6F59
:107B60004F6F506F516F526F536F546F556F566F09
:107B7000576F586F596F5A6F5B6F5C6F5D6F5E6FB9
:107B80005F6F606F616F626F636F646F656F666F69
:107B9000676F686F696F6A6F6B6F6C6F6D6F6E6F19
:107BA0006F6F706F716F726F736F746F756F766FC9
:107BB000776F786F796F7A6F7B6F7C6F7D6F7E6F79
:107BC0007F6F806F816F826F836F846F2B0E856FE5
:107BD000866B7C0E876F3F0E886F200E896F8A6FD1
:107BE0008B6F8C6F8D6F8E6F8F6F906F916F926FA9
:107BF0002D0E936F200E946F540E956F680E966F36
:107C0000690E976F730E986F200E996F6D0E9A6FB5
:107C1000650E9B6F6E0E9C6F750E9D6F200E9E6F96
:107C20009F6FA06FA16FA26FA36FA46FA56FA66FC8
:107C3000A76FA86FA96FAA6FAB6FAC6FAD6FAE6F78
:107C4000AF6FB06FB16FB26FB36FB46FB56FB66F28
:107C5000B76FB86FB96FBA6FBB6FBC6FBD6FBE6FD8
:107C6000BF6FC06FC16FC26FC36FC46FC56FC66F88
:107C7000C76FC86FC96FCA6FCB6FCC6FCD6FCE6F38
:107C8000CF6FD06FD16FD26FD36F7C0ED46FD56BA7
:107C90002B0ED66F2D0ED76FD86FD96FDA6FDB6FC3
:107CA000DC6FDD6FDE6FDF6FE06FE16FE26FE36F60
:107CB000E46FE56F200EE66F530EE76F790EE86F05
:107CC000730EE96F740EEA6F650EEB6F6D0EEC6F5D
:107CD000200EED6F2D0EEE6FEF6FF06FF16FF26F04
:107CE000F36FF46FF56FF66FF76FF86FF96FFA6F68
:107CF000FB6FFC6FFD6FFE6FFF6F0601006F016F82
:107D0000026F036F046F056F066F076F086F096FCF
:107D10000A6F0B6F0C6F0D6F0E6F0F6F106F116F7F
:107D2000126F136F146F156F166F176F186F196F2F
:107D30001A6F1B6F1C6F1D6F1E6F1F6F206F216FDF
:107D4000226F2B0E236F246B7C0E256F500E266F37
:107D50006F0E276F770E286F650E296F720E2A6FD0
:107D6000200E2B6F2C6F2D6F2E6F2F6F306F780EB4
:107D7000316F2D0E326F200E336F500E346F6F0E39
:107D8000356F770E366F650E376F720E386F280EAF
:107D9000396F4F0E3A6F6E0E3B6F2F0E3C6F4F0ECA
:107DA0003D6F660E3E6F3F6F290E406F200E416F94
:107DB000426F436F446F456F466F476F486F496F1F
:107DC0004A6F4B6F4C6F4D6F4E6F7C0E4F6F430E73
:107DD000506F6C0E516F650E526F610E536F720EC5
:107DE000546F4D0E556F650E566F6D0E576F200E0A
:107DF000586F596F5A6F5B6F2D0E5C6F200E5D6F61
:107E0000430E5E6F6C0E5F6F650E606F610E616F8B
:107E1000720E626F200E636F4D0E646F650E656F9C
:107E20006D0E666F6F0E676F720E686F790E696FF9
:107E3000200E6A6F6B6F6C6F6D6F6E6F6F6F706F10
:107E4000716F7C0E726F736B746F530E756F650E6E
:107E5000766F720E776F690E786F610E796F6C0EA8
:107E60007A6F450E7B6F630E7C6F680E7D6F6F0EB1
:107E70007E6F200E7F6F780E806F2D0E816F200E2B
:107E8000826F450E836F630E846F680E856F6F0E71
:107E9000866F200E876F530E886F650E896F720E86
:107EA0008A6F690E8B6F610E8C6F6C0E8D6F200E5A
:107EB0008E6F280E8F6F590E906F650E916F730E37
:107EC000926F2F0E936F4E0E946F6F0E956F200E64
:107ED000966F976F986F996F9A6F9B6F9C6F9D6F5E
:107EE0007C0E9E6F520E9F6F650EA06F730EA16F7A
:107EF000650EA26F740EA36F200EA46FA56FA66F00
:107F0000A76FA86FA96FAA6F2D0EAB6F200EAC6F75
:107F1000270EAD6F430EAE6F500EAF6F550EB06FA4
:107F2000270EB16F520EB26F650EB36F730EB46F42
:107F3000650EB56F740EB66F200EB76FB86FB96F60
:107F4000BA6FBB6FBC6FBD6FBE6FBF6FC06F7C0E73
:107F5000C16FC26BC36F560EC46F650EC56F720ED4
:107F6000C66F730EC76F690EC86F6F0EC96F6E0E46
:107F7000CA6F200ECB6FCC6FCD6FCE6FCF6F2D0E33
:107F8000D06F200ED16F460ED26F690ED36F720E76
:107F9000D46F6D0ED56F770ED66F610ED76F720EE0
:107FA000D86F650ED96F200EDA6F560EDB6F650E37
:107FB000DC6F720EDD6F730EDE6F690EDF6F6F0E9A
:107FC000E06F6E0EE16F200EE26FE36FE46FE56F1E
:107FD000E66FE76FE86FE96FEA6FEB6FEC6F7C0EAF
:107FE000ED6F430EEE6F6F0EEF6F6E0EF06F660E5D
:107FF000F16F690EF26F670EF36F200EF46FF56F7D
:10800000F66FF76FF86FF96F2D0EFA6F200EFB6F9A
:108010004C0EFC6F690EFD6F730EFE6F740EFF6FDA
:10802000200E0701006F430E016F6F0E026F6E0E80
:10803000036F660E046F690E056F670E066F200EE4
:10804000076F530E086F650E096F740E0A6F0B6F82
:10805000690E0C6F6E0E0D6F670E0E6F730E0F6F45
:108060007C0E106F116B126F450E136F146F440E60
:10807000156F750E166F6D0E176F700E186F200E40
:10808000196F1A6F1B6F1C6F1D6F1E6F2D0E1F6FE8
:10809000200E206F440E216F690E226F730E236F26
:1080A000700E246F6C0E256F610E266F790E276F90
:1080B000200E286F430E296F4F0E2A6F6E0E2B6F06
:1080C000660E2C6F690E2D6F670E2E6F200E2F6FB0
:1080D000450E306F316F500E326F720E336F6F0E70
:1080E000346F6D0E356F200E366F376F386F396F06
:1080F0003A6F3B6F7C0E3C6F200E3D6F490E3E6F1A
:108100006E0E3F6F700E406F750E416F740E426FB2
:10811000200E436F446F456F466F476F780E486F70
:108120002D0E496F200E4A6F490E4B6F6E0E4C6F2D
:10813000700E4D6F750E4E6F740E4F6F200E506F98
:10814000280E516F310E526F2F0E536F320E546F37
:10815000290E556F200E566F576F586F596F5A6F13
:108160005B6F5C6F5D6F5E6F7C0E5F6F606B616FEE
:10817000200E626F636F646F656F666F676F686F05
:10818000696F6A6F6B6F6C6F6D6F6E6F6F6F706F13
:10819000716F726F736F746F756F766F776F786FC3
:1081A000796F7A6F7B6F7C6F7D6F7E6F7F6F806F73
:1081B000816F826F836F846F856F866F876F886F23
:1081C000896F8A6F7C0E8B6F200E8C6F4F0E8D6FB8
:1081D000750E8E6F740E8F6F700E906F750E916F9F
:1081E000740E926F200E936F946F956F966F780E4A
:1081F000976F2D0E986F200E996F4F0E9A6F750E18
:108200009B6F740E9C6F700E9D6F750E9E6F740E3B
:108210009F6F200EA06F280EA16F310EA26F2F0E40
:10822000A36F320EA46F290EA56F200EA66FA76F45
:10823000A86FA96FAA6FAB6FAC6FAD6F7C0EAE6FFE
:10824000AF6B2B0EB06F2D0EB16FB26FB36FB46FFB
:10825000B56FB66FB76FB86FB96FBA6FBB6FBC6FE2
:10826000BD6FBE6FBF6FC06FC16FC26FC36FC46F92
:10827000C56FC66FC76FC86FC96FCA6FCB6FCC6F42
:10828000CD6FCE6FCF6FD06FD16FD26FD36FD46FF2
:10829000D56FD66FD76FD86FD96FDA6FDB6FDC6FA2
:1082A000DD6FDE6FDF6FE06FE16FE26FE36FE46F52
:1082B000E56FE66FE76FE86FE96FEA6FEB6FEC6F02
:1082C000ED6FEE6FEF6FF06FF16FF26FF36FF46FB2
:1082D000F56FF66FF76FF86FF96FFA6FFB6FFC6F62
:1082E0002B0EFD6FFE6B0A0E000105EC0FF00D0E5C
:1082F00005EC0FF00401986B98510A0835E3996B6F
:1083000099514E0827E30801006B98C4FFF7026BF0
:108310004F0E016F00016BEC1CF002C000F801C0B1
:10832000FFF7040199510701FF25016E000E0801B6
:108330000021036E01509A0FE96E040E0320EA6ECD
:10834000EFCFFFF70701FF51000105EC0FF004012B
:10835000992BD6D70A0E000105EC0FF00D0E05EC97
:108360000FF00401982BC8D76C0EF66E1B0EF76E3B
:10837000000EF86E0001C5EC3CF0BFEF4AF00401BE
:10838000C151000A000108E0010A31E0030A5AE085
:10839000010AD8B482D0ADD04DA015D0C3C4EAFF35
:1083A000C2C4E9FFF2CFC4F4F29E000EE6EC03F083
:1083B0000A000900F550EE6E0009FBE10401C4BF9C
:1083C000F28E14D00001C3C4EAFFC2C4E9FFF2CFA9
:1083D000C4F4F29E000EFFEC03F00A000900F55011
:1083E000EE6E0009FBE10401C4BFF28E96D04DA2EF
:1083F00015D0C3C4EAFFC2C4E9FFF2CFC4F4F29EB1
:10840000000E19EC04F00A000900F550EE6E0009A8
:10841000FBE10401C4BFF28E14D00001C3C4EAFF23
:10842000C2C4E9FFF2CFC4F4F29E000E36EC04F0B1
:108430000A000900F550EE6E0009FBE10401C4BF1B
:10844000F28E6BD04DA415D0C3C4EAFFC2C4E9FFBD
:10845000F2CFC4F4F29E000E53EC04F00A000900BF
:10846000F550EE6E0009FBE10401C4BFF28E14D09A
:108470000001C3C4EAFFC2C4E9FFF2CFC4F4F29E14
:10848000000E6DEC04F00A000900F550EE6E0009D4
:10849000FBE10401C4BFF28E40D04DA615D0C3C489
:1084A000EAFFC2C4E9FFF2CFC4F4F29E000E87ECEB
:1084B00004F00A000900F550EE6E0009FBE104012A
:1084C000C4BFF28E14D00001C3C4EAFFC2C4E9FFE6
:1084D000F2CFC4F4F29E000EA1EC04F00A000900F1
:1084E000F550EE6E0009FBE10401C4BFF28E15D019
:1084F0000001C3C4EAFFC2C4E9FFF2CFC4F4F29E94
:10850000000EBCEC04F00A000900F550EE6E000904
:10851000FBE10401C4BFF28E00D0000115EF48F06A
:108520000401C15100D0C3C4EAFFC2C4E9FFF2CFC5
:10853000C4F4F29E000E0001BCEC04F00A00090035
:10854000F550EE6E0009FBE10401C4BFF28E00D0CD
:1085500000013DEF48F00401C151000A000101E0B3
:108560002CD01EA015D0C3C4EAFFC2C4E9FFF2CFCD
:10857000C4F4F29E000ECCEC04F00A000900F550A1
:10858000EE6E0009FBE10401C4BFF28E14D00001BD
:10859000C3C4EAFFC2C4E9FFF2CFC4F4F29E000EE6
:1085A000E5EC04F00A000900F550EE6E0009FBE16D
:1085B0000401C4BFF28E15D00001C3C4EAFFC2C4D7
:1085C000E9FFF2CFC4F4F29E000EBCEC04F00A0006
:1085D0000900F550EE6E0009FBE10401C4BFF28E04
:1085E00000D0000165EF48F00401C52D3FD2C22D37
:1085F00085D1C151000A00012BE0010A3DE0030AC8
:108600004FE0010A61E0070AD8B472D0010AD8B479
:1086100083D0030AD8B494D0010AD8B4A5D00F0AE5
:10862000D8B4B6D0010AD8B4C7D0030AD8B4D8D0C9
:10863000010AD8B4E9D0070AD8B4FAD0010AD8B4EC
:108640000BD1030AD8B41CD1010AD8B42DD141D121
:10865000C4C4EAFFC3C4E9FFF2CFC6F4F29E000E21
:10866000FFEC04F00A000900F550EE6E0009FBE192
:108670000401C6BFF28E41D1C4C4EAFFC3C4E9FFFE
:10868000F2CFC6F4F29E000E17EC05F00A000900C6
:10869000F550EE6E0009FBE10401C6BFF28E2DD14C
:1086A000C4C4EAFFC3C4E9FFF2CFC6F4F29E000ED1
:1086B0002FEC05F00A000900F550EE6E0009FBE111
:1086C0000401C6BFF28E19D1C4C4EAFFC3C4E9FFD6
:1086D000F2CFC6F4F29E000E47EC05F00A00090046
:1086E000F550EE6E0009FBE10401C6BFF28E05D124
:1086F000C4C4EAFFC3C4E9FFF2CFC6F4F29E000E81
:108700005FEC05F00A000900F550EE6E0009FBE190
:108710000401C6BFF28EF1D0C4C4EAFFC3C4E9FFAE
:10872000F2CFC6F4F29E000E77EC05F00A000900C5
:10873000F550EE6E0009FBE10401C6BFF28EDDD0FC
:10874000C4C4EAFFC3C4E9FFF2CFC6F4F29E000E30
:108750008FEC05F00A000900F550EE6E0009FBE110
:108760000401C6BFF28EC9D0C4C4EAFFC3C4E9FF86
:10877000F2CFC6F4F29E000EA7EC05F00A00090045
:10878000F550EE6E0009FBE10401C6BFF28EB5D0D4
:10879000C4C4EAFFC3C4E9FFF2CFC6F4F29E000EE0
:1087A000BFEC05F00A000900F550EE6E0009FBE190
:1087B0000401C6BFF28EA1D0C4C4EAFFC3C4E9FF5E
:1087C000F2CFC6F4F29E000ED7EC05F00A000900C5
:1087D000F550EE6E0009FBE10401C6BFF28E8DD0AC
:1087E000C4C4EAFFC3C4E9FFF2CFC6F4F29E000E90
:1087F000EFEC05F00A000900F550EE6E0009FBE110
:108800000401C6BFF28E79D0C4C4EAFFC3C4E9FF35
:10881000F2CFC6F4F29E000E07EC06F00A00090043
:10882000F550EE6E0009FBE10401C6BFF28E65D083
:10883000C4C4EAFFC3C4E9FFF2CFC6F4F29E000E3F
:108840001FEC06F00A000900F550EE6E0009FBE18E
:108850000401C6BFF28E51D0C4C4EAFFC3C4E9FF0D
:10886000F2CFC6F4F29E000E37EC06F00A000900C3
:10887000F550EE6E0009FBE10401C6BFF28E3DD05B
:10888000C4C4EAFFC3C4E9FFF2CFC6F4F29E000EEF
:108890004FEC06F00A000900F550EE6E0009FBE10E
:1088A0000401C6BFF28E29D0C4C4EAFFC3C4E9FFE5
:1088B000F2CFC6F4F29E000E67EC06F00A00090043
:1088C000F550EE6E0009FBE10401C6BFF28E15D033
:1088D0000001C4C4EAFFC3C4E9FFF2CFC6F4F29EAC
:1088E000000E7FEC06F00A000900F550EE6E00095C
:1088F000FBE10401C6BFF28E00D0B7D0C25102081E
:10890000D8A4B3D0C151000A00010EE0010A20E052
:10891000030A32E0010A44E0070A56E0010A68E06F
:10892000030AD8B479D08DD0C4C4EAFFC3C4E9FF28
:10893000F2CFC6F4F29E000EFFEC04F00A0009002C
:10894000F550EE6E0009FBE10401C6BFF28E8DD03A
:10895000C4C4EAFFC3C4E9FFF2CFC6F4F29E000E1E
:1089600047EC05F00A000900F550EE6E0009FBE146
:108970000401C6BFF28E79D0C4C4EAFFC3C4E9FFC4
:10898000F2CFC6F4F29E000E5FEC05F00A0009007B
:10899000F550EE6E0009FBE10401C6BFF28E65D012
:1089A000C4C4EAFFC3C4E9FFF2CFC6F4F29E000ECE
:1089B00077EC05F00A000900F550EE6E0009FBE1C6
:1089C0000401C6BFF28E51D0C4C4EAFFC3C4E9FF9C
:1089D000F2CFC6F4F29E000E8FEC05F00A000900FB
:1089E000F550EE6E0009FBE10401C6BFF28E3DD0EA
:1089F000C4C4EAFFC3C4E9FFF2CFC6F4F29E000E7E
:108A00004FEC06F00A000900F550EE6E0009FBE19C
:108A10000401C6BFF28E29D0C4C4EAFFC3C4E9FF73
:108A2000F2CFC6F4F29E000E67EC06F00A000900D1
:108A3000F550EE6E0009FBE10401C6BFF28E15D0C1
:108A40000001C4C4EAFFC3C4E9FFF2CFC6F4F29E3A
:108A5000000E7FEC06F00A000900F550EE6E0009EA
:108A6000FBE10401C6BFF28E00D06DD2C22DB4D19D
:108A7000C151000A000132E0010A44E0030A56E055
:108A8000010AD8B467D0070AD8B478D0010AD8B49C
:108A900089D0030AD8B49AD0010AD8B4ABD00F0A4F
:108AA000D8B4BCD0010AD8B4CDD0030AD8B4DED033
:108AB000010AD8B4EFD0070AD8B400D1010AD8B45B
:108AC00011D1030AD8B422D1010AD8B433D11F0A74
:108AD000D8B444D1010AD8B455D169D1C4C4EAFF8D
:108AE000C3C4E9FFF2CFC6F4F29E000EFFEC04F01F
:108AF0000A000900F550EE6E0009FBE10401C6BF53
:108B0000F28E69D1C4C4EAFFC3C4E9FFF2CFC6F450
:108B1000F29E000E17EC05F00A000900F550EE6E0B
:108B20000009FBE10401C6BFF28E55D1C4C4EAFFBF
:108B3000C3C4E9FFF2CFC6F4F29E000E2FEC05F09D
:108B40000A000900F550EE6E0009FBE10401C6BF02
:108B5000F28E41D1C4C4EAFFC3C4E9FFF2CFC6F428
:108B6000F29E000E47EC05F00A000900F550EE6E8B
:108B70000009FBE10401C6BFF28E2DD1C4C4EAFF97
:108B8000C3C4E9FFF2CFC6F4F29E000E5FEC05F01D
:108B90000A000900F550EE6E0009FBE10401C6BFB2
:108BA000F28E19D1C4C4EAFFC3C4E9FFF2CFC6F400
:108BB000F29E000E77EC05F00A000900F550EE6E0B
:108BC0000009FBE10401C6BFF28E05D1C4C4EAFF6F
:108BD000C3C4E9FFF2CFC6F4F29E000E8FEC05F09D
:108BE0000A000900F550EE6E0009FBE10401C6BF62
:108BF000F28EF1D0C4C4EAFFC3C4E9FFF2CFC6F4D9
:108C0000F29E000E8FEC06F00A000900F550EE6EA1
:108C10000009FBE10401C6BFF28EDDD0C4C4EAFF47
:108C2000C3C4E9FFF2CFC6F4F29E000EA7EC05F034
:108C30000A000900F550EE6E0009FBE10401C6BF11
:108C4000F28EC9D0C4C4EAFFC3C4E9FFF2CFC6F4B0
:108C5000F29E000EBFEC05F00A000900F550EE6E22
:108C60000009FBE10401C6BFF28EB5D0C4C4EAFF1F
:108C7000C3C4E9FFF2CFC6F4F29E000ED7EC05F0B4
:108C80000A000900F550EE6E0009FBE10401C6BFC1
:108C9000F28EA1D0C4C4EAFFC3C4E9FFF2CFC6F488
:108CA000F29E000EA7EC06F00A000900F550EE6EE9
:108CB0000009FBE10401C6BFF28E8DD0C4C4EAFFF7
:108CC000C3C4E9FFF2CFC6F4F29E000EEFEC05F04C
:108CD0000A000900F550EE6E0009FBE10401C6BF71
:108CE000F28E79D0C4C4EAFFC3C4E9FFF2CFC6F460
:108CF000F29E000E07EC06F00A000900F550EE6E39
:108D00000009FBE10401C6BFF28E65D0C4C4EAFFCE
:108D1000C3C4E9FFF2CFC6F4F29E000E1FEC06F0CA
:108D20000A000900F550EE6E0009FBE10401C6BF20
:108D3000F28E51D0C4C4EAFFC3C4E9FFF2CFC6F437
:108D4000F29E000EBFEC06F00A000900F550EE6E30
:108D50000009FBE10401C6BFF28E3DD0C4C4EAFFA6
:108D6000C3C4E9FFF2CFC6F4F29E000E4FEC06F04A
:108D70000A000900F550EE6E0009FBE10401C6BFD0
:108D8000F28E29D0C4C4EAFFC3C4E9FFF2CFC6F40F
:108D9000F29E000E67EC06F00A000900F550EE6E38
:108DA0000009FBE10401C6BFF28E15D00001C4C466
:108DB000EAFFC3C4E9FFF2CFC6F4F29E000E7FECD7
:108DC00006F00A000900F550EE6E0009FBE104010F
:108DD000C6BFF28E00D0B7D0C2510208D8A4B3D01B
:108DE000C151000A00010EE0010A20E0030A32E04E
:108DF000010A44E0070A56E0010A68E0030AD8B411
:108E000079D08DD0C4C4EAFFC3C4E9FFF2CFC6F461
:108E1000F29E000EFFEC04F00A000900F550EE6E21
:108E20000009FBE10401C6BFF28E8DD0C4C4EAFF85
:108E3000C3C4E9FFF2CFC6F4F29E000E47EC05F082
:108E40000A000900F550EE6E0009FBE10401C6BFFF
:108E5000F28E79D0C4C4EAFFC3C4E9FFF2CFC6F4EE
:108E6000F29E000E5FEC05F00A000900F550EE6E70
:108E70000009FBE10401C6BFF28E65D0C4C4EAFF5D
:108E8000C3C4E9FFF2CFC6F4F29E000E77EC05F002
:108E90000A000900F550EE6E0009FBE10401C6BFAF
:108EA000F28E51D0C4C4EAFFC3C4E9FFF2CFC6F4C6
:108EB000F29E000E8FEC05F00A000900F550EE6EF0
:108EC0000009FBE10401C6BFF28E3DD0C4C4EAFF35
:108ED000C3C4E9FFF2CFC6F4F29E000E4FEC06F0D9
:108EE0000A000900F550EE6E0009FBE10401C6BF5F
:108EF000F28E29D0C4C4EAFFC3C4E9FFF2CFC6F49E
:108F0000F29E000E67EC06F00A000900F550EE6EC6
:108F10000009FBE10401C6BFF28E15D00001C4C4F4
:108F2000EAFFC3C4E9FFF2CFC6F4F29E000E7FEC65
:108F300006F00A000900F550EE6E0009FBE104019D
:108F4000C6BFF28E00D0C3C401F0C4C402F0000159
:108F5000000C0401C06B040EEA6E980EE96E060167
:108F60000F6B116B280E106F000187EC0FF0E5EC12
:108F700016F07A0EF66E1A0EF76E000EF86E100EE0
:108F800005012A6F0001A8EC1BF0EA6A310EE96EB8
:108F9000B2EC3CF0EA6A230EE96EB2EC3CF00A0E49
:108FA0009EA8FED7AD6E0D0E9EA8FED7AD6E920E9A
:108FB000F66E1A0EF76E000EF86E0E0E05012A6F91
:108FC0000001A8EC1BF0AC0EF66E1A0EF76E000E48
:108FD000F86EC5EC3CF0A20EF66E1A0EF76E000E9F
:108FE000F86E040E05012A6F0001A8EC1BF0B60E06
:108FF000F66E1A0EF76E000EF86EC5EC3CF00A0E17
:109000009EA8FED7AD6E0D0E9EA8FED7AD6E0401D4
:10901000C06BC051070824E3C0C4C1F4040EC36F81
:10902000980EC26F0001BFEF41F0040E0601106FF1
:10903000980E0F6F000125EC12F001520EE0040EA5
:10904000EA6E980EE96EB2EC3CF00A0E9EA8FED7CE
:10905000AD6E0D0E9EA8FED7AD6E0401C02BD9D704
:10906000C06BC051070824E3C0C4C1F4040EC36F31
:10907000980EC26F000190EF42F0040E0601106FCF
:10908000980E0F6F000125EC12F001520EE0040E55
:10909000EA6E980EE96EB2EC3CF00A0E9EA8FED77E
:1090A000AD6E0D0E9EA8FED7AD6E0401C02BD9D7B4
:1090B000C06BC051070824E3C0C4C1F4040EC36FE1
:1090C000980EC26F0001ABEF42F0040E0601106F64
:1090D000980E0F6F000125EC12F001520EE0040E05
:1090E000EA6E980EE96EB2EC3CF00A0E9EA8FED72E
:1090F000AD6E0D0E9EA8FED7AD6E0401C02BD9D764
:1091000050C0C1F4010EC26F040EC46F980EC36F3D
:10911000010EC56F0001F4EC42F0C00EF66E1A0E9F
:10912000F76E000EF86E090E05012A6F0001A8EC1B
:109130001BF0040EEA6E980EE96EB2EC3CF02C0EB9
:109140009EA8FED7AD6E51C0C1F4010E0401C26FDE
:10915000040EC46F980EC36FC56B0001F4EC42F0AF
:10916000CE0EF66E1A0EF76E000EF86E0A0E0501A0
:109170002A6F0001A8EC1BF0040EEA6E980EE96E4F
:10918000B2EC3CF02C0E9EA8FED7AD6E52C0C1F4DE
:10919000020E0401C26F040EC46F980EC36FC56B3C
:1091A0000001F4EC42F0DC0EF66E1A0EF76E000EC3
:1091B000F86E0A0E05012A6F0001A8EC1BF0040EE0
:1091C000EA6E980EE96EB2EC3CF00A0E9EA8FED74D
:1091D000AD6E0D0E9EA8FED7AD6E54C0C1F4020E4A
:1091E0000401C26F040EC46F980EC36F010EC56FE9
:1091F0000001F4EC42F0EC0EF66E1A0EF76E000E63
:10920000F86E090E05012A6F0001A8EC1BF0040E90
:10921000EA6E980EE96EB2EC3CF02C0E9EA8FED7DA
:10922000AD6E55C0C1F4010E0401C26F040EC46FCF
:10923000980EC36FC56B0001F4EC42F0FA0EF66EA7
:109240001A0EF76E000EF86E0A0E05012A6F000165
:10925000A8EC1BF0040EEA6E980EE96EB2EC3CF03E
:109260002C0E9EA8FED7AD6E56C0C1F4020E0401AE
:10927000C26F040EC46F980EC36FC56B0001F4EC8F
:1092800042F0080EF66E1B0EF76E000EF86E0A0E18
:1092900005012A6F0001A8EC1BF0040EEA6E980E7F
:1092A000E96EB2EC3CF00A0E9EA8FED7AD6E0D0E34
:1092B0009EA8FED7AD6E180EF66E1B0EF76E000E52
:1092C000F86EC5EC3CF0C2EF4AF00401996B986B64
:1092D000996B986B9951030842E398510F0B9B6F60
:1092E0009C6B9B531EE19C531CE10A0E9EA8FED76B
:1092F000AD6E0D0E9EA8FED7AD6E99C4ADF4370EBF
:10930000AE6F000148EC1CF098C4ADF4370E0401B8
:10931000AE6F000148EC1CF0200E9EA8FED7AD6E8B
:109320000401F2CF9BF4F29E99C4AAFF98C4A9FF4E
:10933000A69CA69EA680A8509BBFF28E9A6F9AC448
:10934000ADF4370EAE6F000148EC1CF0200E9EA865
:10935000FED7AD6E0401982BD8B4992BBBD72E0E37
:10936000F66E1B0EF76E000EF86E0001C5EC3CF0B9
:1093700021EF4BF0036ADC518A0FE96E000E0320E7
:10938000EA6EEFCF2CF50501010E0001DC25050189
:109390002E6F2F6F510E306F0001C1EC1BF000C01B
:1093A000DCF0DB51DC5D01E1DD9105012CC501F054
:1093B0000001000C0401986B0001DDA10AD0DADF86
:1093C00001C098F4010E0401CC6F0001B9EC0FF05C
:1093D000F4D7000C0401986B986B9851020821E3B4
:1093E000036A9851AE0FE96E020E0320EA6EEF6A2F
:1093F000036A9851B30F016E020E032203C09AF460
:10940000036A9851BD0FE96E020E0320EA6EEFCF9A
:109410009BF49AC4EAFF01C0E9FF9BC4EFFF982BBD
:10942000DCD7996B0001D5EC17F00201AD6B0001A0
:10943000DD99DD9BDD9D04013D6B3C6B3DC441F43A
:109440003CC440F441C43FF440C43EF4036A02010A
:10945000AD51B30FE96E020E0320EA6EEFCF99F41F
:1094600099C49AF4060E04019B6F0001B7EC1AF040
:10947000C9EF4BF04DA02CD0880EF66E1C0EF76E87
:10948000000EF86E110E05012A6F0001A8EC1BF00A
:1094900083C4ADF4570E0401AE6F000148EC1CF01C
:1094A0002F0E9EA8FED7AD6E83C49FF41B0E040141
:1094B000A06F0001F7EC20F0290E9EA8FED7AD6E3C
:1094C0000A0E9EA8FED7AD6E0D0E9EA8FED7AD6EFD
:1094D0000F0E0401835DF00FD8B095D1100F00017D
:1094E00006EF4CF0A40EF66E1C0EF76E000EF86E32
:1094F0000F0E05012A6F0001A8EC1BF0EA6A1F0E8F
:10950000E96EB2EC3CF00A0E9EA8FED7AD6E0D0ED1
:109510009EA8FED7AD6EB80EF66E1C0EF76E000E4E
:10952000F86E0E0E05012A6F0001A8EC1BF0D20E9A
:10953000F66E1C0EF76E000EF86EC5EC3CF0C80E11
:10954000F66E1C0EF76E000EF86E040E05012A6F03
:109550000001A8EC1BF0DC0EF66E1C0EF76E000E80
:10956000F86EC5EC3CF00A0E9EA8FED7AD6E0D0E4F
:109570009EA8FED7AD6E040146D1DAEF3CF004019F
:1095800042D1E7D404013FD113EC2EF004013BD1CA
:10959000040EEA6E840EE96EF2CF98F4F29E000E8D
:1095A00067EC07F00A000900F550EE6E0009FBE1D8
:1095B000040198BFF28E040EA06F840E9F6F00010D
:1095C0002CEC22F0030EAA6EE00EA96EA86AA69CEF
:1095D000A69EA684F250006EF29E0F01550EA76E55
:1095E000AA0EA76EA682A6B2FED7A6940050F212CB
:1095F000040EEA6E840EE96EF2CF98F4F29E000E2D
:1096000000017FEC07F00A000900F550EE6E00093A
:10961000FBE1040198BFF28E040EA06F840E9F6FD1
:1096200000012CEC22F0080E0401986FFA0ECC6FAA
:109630000001B9EC0FF00401982FF8D7FF00E3D038
:1096400044D60401E0D00401DED0B4DE896BEA6ABE
:109650008A0EE96E06010F6B116B510E106F00013F
:1096600087EC0FF0DB6BDBC0DCF0DD919D8A040141
:10967000CAD0040EEA6E840EE96E06010F6B116B00
:10968000140E106F000187EC0FF0040E0401A06FA0
:10969000840E9F6F00012CEC22F09D9A8BDE9EECD5
:1096A0001BF00401B0D0E60EF66E1C0EF76E000E35
:1096B000F86EC5EC3CF00401A6D0040EEA6E840EF0
:1096C000E96E06010F6B116B140E106F000187EC31
:1096D0000FF0040EEA6E840EE96EF2CF98F4F29E5B
:1096E000000E7FEC07F00A000900F550EE6E00094D
:1096F000FBE1040198BFF28E040EA06F840E9F6FF1
:1097000000012CEC22F0080E0401986FFA0ECC6FC9
:109710000001B9EC0FF00401982FF8D7FF0073D0C7
:10972000040EEA6E840EE96E06010F6B116B140EC7
:10973000106F000187EC0FF0040EEA6E840EE96EE4
:10974000F2CF98F4F29E000E97EC07F00A000900A1
:10975000F550EE6E0009FBE1040198BFF28E040E95
:10976000A06F840E9F6F00012CEC22F0080E040104
:10977000986FFA0ECC6F0001B9EC0FF00401982F2E
:10978000F8D7210E9F6F010EA06F000139EC21F078
:1097900021D60401A06BA16BA26BA46BA36BA66B7B
:1097A000A56B00016AEC23F00401A06BA16BA26B16
:1097B000A46BA36BA66BA56B00017DEC22F00401EA
:1097C00022D01E801EB208D07E868A0EAF6E000E9A
:1097D0007F6EA60EAC6E07D07E86400EAF6E030E77
:1097E0007F6EA60EAC6E04010ED01E901E927E8679
:1097F000400EAF6E030E7F6EA60EAC6E040103D05A
:10980000040101D00401000169EF4CF0F2CF0DF02A
:10981000F29EE824F76AF736370FF66E980EF722B5
:10982000000EF86EFB6E0A00F550FA6E0800F55057
:109830000DBEF28EF96EE4947A9582958895909596
:10984000409646964A967296BA9620970098A696A3
:109850000498C297EA970401826B0001DDB701D03A
:1098600038D0BDEF20F001C082F402012351040181
:10987000825D0DE382510201295DD8B002D004015E
:1098800006D082C483F4000164EF24F022D00201E8
:1098900024510401825D0DE3825102012A5DD8B09A
:1098A00002D0040106D082C483F400017DEF3CF0B5
:1098B00010D0020125510401825D0CE382510201A6
:1098C0002B5DD8B002D0040105D082C483F400011E
:1098D000D1D50401000177EF58F033C537F532C513
:1098E00036F537C503F0050136C5E9FF37C5EAFF90
:1098F000EF5230E035C539F534C538F539C503F0D8
:1099000038C5E9FF39C5EAFFEF520AE13251365D49
:10991000006E33513759036E00C001F023D010D0D0
:1099200036C5E9FF37C5EAFFEFCF3AF539C503F091
:1099300038C5E9FF39C5EAFFEF503A5D01E104D0CF
:10994000382BD8B4392BDAD7362BD8B4372B0001C3
:10995000C8D705013251365D006E33513759036E59
:1099600000C001F000010AEF4DF033C537F532C5F4
:1099700036F537C503F0050136C5E9FF37C5EAFFFF
:10998000EF522AE035C539F534C538F539C503F04D
:1099900038C5E9FF39C5EAFFEF5218E036C5E9FFDF
:1099A00037C5EAFFEFCF3AF539C503F038C5E9FF0F
:1099B00039C5EAFFEF503A5D05E136C501F037C51C
:1099C00002F00DD0382BD8B4392BE0D7362BD8B4D1
:1099D000372B0001CED70501000E016E026E00018B
:1099E0002BEF4DF005012A512B1104E02BC503F09C
:1099F0002A5103D019C003F018502E6F03C02FF561
:109A00002FC533F52EC532F52DC535F52CC534F5EA
:109A1000000163D7015005012E27000E2F232FC50B
:109A200003F02EC5E9FF2FC5EAFFEF520AE118C087
:109A3000E9FF19C0EAFF200EEF6E000E016E026E04
:109A400027D02FC533F52EC532F52DC535F52CC5DC
:109A500034F500018AD702C031F501C030F531C5B7
:109A600003F0050130C5E9FF31C5EAFFEF5208E018
:109A700030C5E9FF31C5EAFFEF6A302BD8B4312B8E
:109A800031C519F030C518F02EC501F02FC502F010
:109A90000001000C06010FC6E9FF10C6EAFFEFCF78
:109AA00013F612C603F011C6E9FF12C6EAFFEF5023
:109AB000135D48E010C603F00FC6E9FF10C6EAFFC9
:109AC000EFCF13F61351400803E213515A0806E290
:109AD000135160084CE213517A0849E312C603F0AF
:109AE00011C6E9FF12C6EAFFEFCF13F61351400883
:109AF00003E213515A0806E21351600838E2135189
:109B00007A0835E30FC6E9FF10C6EAFFEFCF13F678
:109B100012C603F011C6E9FF12C6EAFF200EEF24B9
:109B2000135D10E011C6E9FF12C6EAFFEFCF13F68E
:109B300010C603F00FC6E9FF10C6EAFF200EEF249F
:109B4000135D15E110C603F00FC6E9FF10C6EAFF6A
:109B5000EF5203E1000E016E1FD010C603F00F514B
:109B60000F2BD8B4102B112BD8B4122B94D710C6AE
:109B700003F00FC6E9FF10C6EAFFEFCF13F612C6D7
:109B800003F011C6E9FF12C6EAFFEF50135D02E2CF
:109B9000FF0E01D0010E016E0001000C006A016A87
:109BA00006011651D89017B100260032013217B3C2
:109BB00000260032013217B500260032013217B7F5
:109BC00000260032013217B900260032013217BBDD
:109BD00000260032013217BD00260032013217BFC5
:109BE000002600320132000164EF4EF00601146BD2
:109BF000126B0A0E136F116B0F51101103E1000E5F
:109C0000016EC3D01451142B036A0F25E96E105155
:109C10000320EA6EEFCF15F615512D080DE1010E68
:109C2000126F1451142B036A0F25E96E1051032093
:109C3000EA6EEFCF15F60DD015512B080AE114513D
:109C4000142B036A0F25E96E10510320EA6EEFCF43
:109C500015F615512F08D8B090D015513908D8A055
:109C60008CD01551300821E1036A14510F25E96E9B
:109C700010510320EA6EEF5078080AE0036A14518D
:109C80000F25E96E10510320EA6EEF5058080DE1E0
:109C9000100E136F142B1451142B036A0F25E96E49
:109CA00010510320EA6EEFCF15F613510A081DE19B
:109CB00015512F0819E21551390816E30A0E166FCF
:109CC00011C617F600016AD7300E0601155D012492
:109CD000116F1451142B036A0F25E96E10510320E4
:109CE000EA6EEFCF15F6E4D748D01351100845E1DE
:109CF0001551600806E215517A0803E31551DF0B90
:109D000001D01551156F15512F0803E2155139086F
:109D100006E21551400831E2155146082EE315516F
:109D20002F080CE21551390809E31139166FF00EAE
:109D30001617300E155D1625116F09D01139166FE3
:109D4000F00E1617410E155D0A0F1625116F1451EE
:109D5000142B036A0F25E96E10510320EA6EEFCF32
:109D600015F61551600806E215517A0803E31551FE
:109D7000DF0B01D01551156FC6D7122D04D013512A
:109D80000A0801E1116D11C601F00001000C050186
:109D90004C6B440E4D6F690E4E6F610E4F6F670E28
:109DA000506F516B526B536B546B556B566B576BBB
:109DB000586B596B5A6B500E5B6F6F0E5C6F770E62
:109DC0005D6F650E5E6F720E5F6F606B616B626BD5
:109DD000636B646B656B666B676B686B520E696F68
:109DE000650E6A6F730E6B6F650E6C6F740E6D6F20
:109DF0006E6B6F6B706B716B726B736B746B756B7F
:109E0000766B490E776F6E0E786F700E796F750EE8
:109E10007A6F740E7B6F7C6B7D6B7E6B7F6B806B60
:109E2000816B826B836B846B450E856F866F440EEE
:109E3000876F750E886F6D0E896F700E8A6F8B6BD2
:109E40008C6B8D6B8E6B8F6B906B916B926B430EEB
:109E5000936F6F0E946F6E0E956F660E966F690E10
:109E6000976F670E986F996B9A6B9B6B9C6B9D6B52
:109E70009E6B9F6BA06B4F0EA16F750EA26F740E41
:109E8000A36F700EA46F750EA56F740EA66FA76BEF
:109E9000A86BA96BAA6BAB6BAC6BAD6BAE6B540EC6
:109EA000AF6F750EB06F6E0EB16FB26F650EB36FA0
:109EB0006C0EB46FB56BB66BB76BB86BB96BBA6B36
:109EC000BB6BBC6B560EBD6F650EBE6F720EBF6F67
:109ED000730EC06F690EC16F6F0EC26F6E0EC36FCF
:109EE000C46BC56BC66BC76BC86BC96BCA6B430EC3
:109EF000CB6F6C0ECC6F650ECD6F610ECE6F720E98
:109F0000CF6F4D0ED06F650ED16F6D0ED26FD36BCC
:109F1000D46BD56BD66BD76BD86B530ED96F650EE0
:109F2000DA6F720EDB6F690EDC6F610EDD6F6C0E27
:109F3000DE6F450EDF6F630EE06F680EE16F6F0E30
:109F4000E26FE36BE46BE56BE66BE76BE86BE96B89
:109F5000EA6BEB6BEC6BED6BEE6BEF6BF06BF16B3D
:109F6000F26BF36BF46B590EF56F650EF66F730EB3
:109F7000F76FF86BF96B4E0EFA6F6F0EFB6FFC6BA1
:109F8000FD6BFE6B4F0EFF6F6E0E0601006F016BD7
:109F9000026B036B4F0E046F660E056F066F076B47
:109FA000086B530E096F6C0E0A6F6F0E0B6F770EF6
:109FB0000C6F0D6B0E6B050EEA6E2E0EE96E0F6BBD
:109FC000116B1E0E106F000187EC0FF0DD852BC5A5
:109FD00010F62AC50FF625EC12F0010E015CF60F03
:109FE000D8B0ECD20A0FEBEF52F005012AC5E9FF19
:109FF0002BC5EAFFEF503F080BE1100E06010F6F73
:10A000000001BCEC16F0010E06010E6F0001DD959B
:10A010000001D4D22BC510F62AC50FF6050E060195
:10A02000126F4D0E116F000135DD015252E12DC549
:10A0300010F62CC50FF625EC12F0015231E02DC5BB
:10A0400010F62CC50FF6050E0601126FFF0E116FEC
:10A05000000120DD01520BE14D80120E06010F6F51
:10A060000001BCEC16F0050E06010E6F17D02DC5D1
:10A0700010F62CC50FF6060E0601126F040E116FB6
:10A08000000108DD01520BE14D90120E06010F6F29
:10A090000001BCEC16F0050E06010E6F000119D090
:10A0A0004D90010809E1820EF66E1B0EF76E000E50
:10A0B000F86EC5EC3CF008D0900EF66E1B0EF76EF5
:10A0C000000EF86EC5EC3CF0DD95050E06010E6F36
:10A0D000000174D22BC510F62AC50FF6050E060135
:10A0E000126F5B0E116F0001D5DC015254E12DC5DA
:10A0F00010F62CC50FF625EC12F0015233E02DC5F9
:10A1000010F62CC50FF6050E0601126FFF0E116F2B
:10A110000001C0DC01520CE184A806D0020E060149
:10A120000F6F0001BCEC16F0080E06010E6F18D080
:10A130002DC510F62CC50FF6060E0601126F040E83
:10A14000116F0001A7DC01520CE184B806D0020EA9
:10A1500006010F6F0001BCEC16F0080E06010E6F31
:10A16000000118D084A809D0A00EF66E1B0EF76E61
:10A17000000EF86EC5EC3CF008D0B00EF66E1B0E6B
:10A18000F76E000EF86EC5EC3CF0080E06010E6F7F
:10A190000001DD956BD02BC510F62AC50FF6050E14
:10A1A0000601126F690E116F000174DC01520AE1A1
:10A1B000180E06010F6F0001BCEC16F0060E06012A
:10A1C0000E6F55D02BC510F62AC50FF6050E0601E9
:10A1D000126F770E116F00015DDC015247E12DC552
:10A1E00010F62CC50FF625EC12F001521CE02DC51F
:10A1F00010F62CC50FF6FADC01C04CF505014C53E6
:10A2000010E04C5102080DE3030E4C25FF0F4C6F7C
:10A210004CC50FF60001BCEC16F00B0E06010E6FDC
:10A22000050125D0000188BD09D0C00EF66E1B0EB9
:10A23000F76E000EF86EC5EC3CF013D088B309D071
:10A24000D40EF66E1B0EF76E000EF86EC5EC3CF0E9
:10A2500008D0E80EF66E1B0EF76E000EF86EC5EC19
:10A260003CF00B0E06010E6F0001DD9505010001AB
:10A27000A5D12BC510F62AC50FF6050E0601126FE3
:10A28000850E116F000106DC01520AE1140E060171
:10A290000F6F0001BCEC16F0060E06010E6FF7D032
:10A2A0002BC510F62AC50FF6050E0601126F930E88
:10A2B000116F00014AEC4DF001520AE1110E060146
:10A2C0000F6F0001BCEC16F0060E06010E6FDFD01A
:10A2D0002BC510F62AC50FF6050E0601126FA10E4A
:10A2E000116F00014AEC4DF001523FE12DC510F60F
:10A2F0002CC50FF625EC12F001521CE02DC510F60E
:10A300002CC50FF673DC01C04CF505014C5310E071
:10A310004C5102080DE3070E4C25FF0F4C6F4CC546
:10A320000FF60001BCEC16F00C0E06010E6F0501D5
:10A330001BD0000188BF08D0F80EF66E1B0EF76E1A
:10A34000000EF86EC5EC3CF088B108D0080EF66E31
:10A350001C0EF76E000EF86EC5EC3CF00C0E0601FC
:10A360000E6F0001DD95050192D02BC510F62AC5B0
:10A370000FF6050E0601126FAF0E116F00014AECC9
:10A380004DF00152D8A482D02DC510F62CC50FF681
:10A3900025EC12F00152D8B479D02DC510F62CC599
:10A3A0000FF6050E0601126FFF0E116F00014AEC49
:10A3B0004DF0015223E11E801E921E847E868A0E7D
:10A3C000AF6E000E7F6EA60EAC6E180EF66E1C0EF3
:10A3D000F76E000EF86EC5EC3CF0DD950E0E060132
:10A3E0000F6F0001BCEC16F00E0E06010F6F00019E
:10A3F000BCEC16F00D0E06010E6F49D02DC510F6FF
:10A400002CC50FF6060E0601126F090E116F000122
:10A410004AEC4DF0015223E11E801E821E847E868E
:10A42000400EAF6E030E7F6EA60EAC6E300EF66E53
:10A430001C0EF76E000EF86EC5EC3CF00E0E060119
:10A440000F6F0001BCEC16F00E0E06010F6F00013D
:10A45000BCEC16F0DD950D0E06010E6F18D02DC563
:10A4600010F62CC50FF6060E0601126F040E116FC2
:10A4700000014AEC4DF0015209E11E901E927E86C9
:10A48000400EAF6E030E7F6EA60EAC6E060100018D
:10A4900095D02BC510F62AC50FF6050E0601126FD2
:10A4A000BD0E116F00014AEC4DF001520AE10F0E92
:10A4B00006010F6F0001BCEC16F00A0E06010E6FCC
:10A4C00000017CD02BC510F62AC50FF6050E06013B
:10A4D000126FCB0E116F00014AEC4DF001520AE1F0
:10A4E000130E06010F6F0001BCEC16F0040E0601FE
:10A4F0000E6F000163D02BC510F62AC50FF6050EAE
:10A500000601126FD90E116F00014AEC4DF0015295
:10A5100054E12DC510F62CC50FF625EC12F00152B2
:10A5200033E02DC510F62CC50FF6050E0601126F8F
:10A53000F50E116F00014AEC4DF001520BE14D8414
:10A54000120E06010F6F0001BCEC16F0030E06019F
:10A550000E6F18D02DC510F62CC50FF6060E06018D
:10A56000126F040E116F00014AEC4DF001520BE125
:10A570004D94120E06010F6F0001BCEC16F0030E95
:10A5800006010E6F000119D04D94010809E1480E33
:10A59000F66E1C0EF76E000EF86EC5EC3CF008D09F
:10A5A0005E0EF66E1C0EF76E000EF86EC5EC3CF0FB
:10A5B000DD95030E06010E6F000100D006010E535B
:10A5C00004E0010E016E04D003D0000E016E00D035
:10A5D0000001F4EF53F0F2CF0DF0F29EE824F76A99
:10A5E000F736010FF66EA60EF722000EF86EFB6E20
:10A5F0000A00F550FA6E0800F5500DBEF28EF96EA5
:10A60000EA9FBCA5BCA514A0D4A072A292A4C4A425
:10A61000BCA5F6A40501236B226B200E246F0D0E42
:10A62000256F266B296B040EEA6E820EE96E060119
:10A630000F6B116B500E106F000187EC0FF0040EC2
:10A64000EA6ED20EE96E06010F6B116B140E106FDD
:10A65000000187EC0FF0040EEA6EE60EE96E0601CB
:10A660000F6B116B3C0E106F000187EC0FF0BAEC12
:10A6700049F001C082F404018251200803E0D25164
:10A680003E0807E10001BAEC49F001C082F4F3D7BB
:10A69000040182510D0803E100018907CCD00501B6
:10A6A000296B036A2951820FE96E040E0320EA6EBA
:10A6B000EF500D081FE029514F0801E3292B00013D
:10A6C000DDA115D0036A05012951820F016E040E28
:10A6D000032201C02AF503C02BF50001BAEC49F0B2
:10A6E0002BC5EAFF2AC5E9FF01C0EFFF01D0A3D0C7
:10A6F0000501D7D7000189070501292B036A2951D4
:10A70000820FE96E040E0320EA6EEF6A040E060162
:10A71000106F820E0F6F000125EC12F00152D8B4B9
:10A720008AD0040E05012B6F820E2A6F050E2D6F45
:10A73000240E2C6F0001F2EC4CF002C023F501C096
:10A7400022F50501225302E123535DE0820E225DD2
:10A750002A6F040E23592B6F2B5355E12A511208EF
:10A7600052E3040EEA6ED20EE96E23C5E2FF22C563
:10A77000E1FFE752E6CFEEFFFCE12B6B2A6B050E03
:10A780002D6F240E2C6F0001F2EC4CF002C023F56B
:10A7900001C022F50501225302E123531AE023C52B
:10A7A00010F622C50FF6000125EC12F001503A0810
:10A7B000D8B002D005010DD0040EEA6EE60EE96EA7
:10A7C00023C5E2FF22C5E1FFE752E6CFEEFFFCE141
:10A7D0000501040E2B6FD20E2A6F040E2D6FE60EAC
:10A7E0002C6F0001C7EF4EF0012C0CD0DDA509D075
:10A7F000DD95440EF66E1B0EF76E000EF86EC5EC7E
:10A800003CF019D005013E0E9EA8FED7AD6E040E99
:10A81000EA6E820EE96E0001B2EC3CF05D0EF66E5F
:10A820001B0EF76E000EF86E0D0E05012A6F00016B
:10A83000A8EC1BF0DD957DEF58F00401826B4DA074
:10A8400031D00001DDA32DD0FC0EF66E1C0EF76E8C
:10A85000000EF86EC5EC3CF0DDA323D07BEC1BF0C2
:10A8600001C082F482C4ADF4570E0401AE6F000142
:10A8700048EC1CF0200E9EA8FED7AD6E0401823D70
:10A880000ED00101205301E020070A0E9EA8FED73A
:10A89000AD6E0D0E9EA8FED7AD6E000102D0000178
:10A8A000DBD70401000183EF58F0F86AD09E078ED1
:10A8B000EA6AE96A700ED36E400E9B6ED3507E86B4
:10A8C000400EAF6E030E7F6EA60EAC6E900EAB6E9A
:10A8D0007C868A0E6F6E000E7D6EA60E6C6E900EDC
:10A8E0006B6E1E6A886B896BDB6BDC6BDD91DD93B5
:10A8F00001011E6B1F6B206B0001DD950201206BB7
:10A900001F6B226B216B0001DD970201AD6B04010F
:10A910003D6B3C6B3F6B3E6B416B406B0001DD99C7
:10A92000DD9BDD9DDD9FC150C00B0F09C16E070E81
:10A93000B46E186A196A200E1F6E200E206E200E4B
:10A94000216E200E226E200E236E560E246E300EC7
:10A95000256E310E266E2E0E276E300E286E300EAE
:10A96000296E2E0E2A6E310E2B6E310E2C6E2D6A34
:10A97000200E316E200E326E550E336E580E346E30
:10A98000480E356E440E366E200E376E430E386E0E
:10A99000720E396E6F0E3A6E730E3B6E730E3C6E16
:10A9A000700E3D6E6F0E3E6E690E3F6E6E0E406E07
:10A9B000740E416E426A300E436E390E446E2D0E97
:10A9C000456E4A0E466E750E476E6E0E486E2D0E23
:10A9D000496E310E4A6E300E4B6E4C6A0201236B8B
:10A9E0000B0E246F0F0E256F1F0E266F276B286B23
:10A9F0000A0E296F0E0E2A6F1E0E2B6F210E2C6F62
:10AA00002D6B2E6B200E2F6F200E306F200E316FAE
:10AA1000200E326F200E336F200E346F200E356FF4
:10AA2000200E366F200E376F200E386F200E396FD4
:10AA3000200E3A6F200E3B6F200E3C6F200E3D6FB4
:10AA4000200E3E6F200E3F6F406B200E416F200E98
:10AA5000426F200E436F200E446F200E456F200E74
:10AA6000466F200E476F200E486F200E496F200E54
:10AA70004A6F200E4B6F200E4C6F200E4D6F200E34
:10AA80004E6F200E4F6F200E506F200E516F526B85
:10AA9000200E536F200E546F200E556F490E566FC7
:10AAA0006E0E576F700E586F750E596F740E5A6F89
:10AAB000200E5B6F310E5C6F200E5D6F4D0E5E6F72
:10AAC000650E5F6F6E0E606F750E616F200E626FA8
:10AAD000200E636F646B200E656F200E666F200E74
:10AAE000676F490E686F6E0E696F700E6A6F750E34
:10AAF0006B6F740E6C6F200E6D6F320E6E6F200ECA
:10AB00006F6F4D0E706F650E716F6E0E726F750EFA
:10AB1000736F200E746F200E756F766B200E776F3B
:10AB2000200E786F200E796F520E7A6F470E7B6F72
:10AB3000420E7C6F480E7D6F560E7E6F200E7F6F2B
:10AB40004F0E806F750E816F740E826F200E836FB3
:10AB5000500E846F6F0E856F730E866F200E876F99
:10AB6000886B200E896F200E8A6F200E8B6F530E1C
:10AB70008C6F790E8D6F730E8E6F740E8F6F650EE6
:10AB8000906F6D0E916F200E926F4D0E936F650E4C
:10AB9000946F6E0E956F750E966F200E976F200E48
:10ABA000986F200E996F9A6B200E9B6F200E9C6FF2
:10ABB000200E9D6F530E9E6F740E9F6F610EA06FDF
:10ABC0006E0EA16F640EA26F620EA36F790EA46F5A
:10ABD000200EA56F4D0EA66F6F0EA76F640EA86FA7
:10ABE000650EA96F200EAA6F200EAB6FAC6BAE6B1B
:10ABF000AF6BB06BB16BB26BB36BB46BB56BB66B69
:10AC0000B76B050EB86F040EB96F030EBA6F030E63
:10AC1000BB6F030EBC6FBD6BBE6BBF6BC06BC16BFC
:10AC2000200EC26F200EC36F200EC46F200EC56FA2
:10AC3000200EC66F200EC76F200EC86F590EC96F49
:10AC4000650ECA6F730ECB6F200ECC6F200ECD6FCA
:10AC5000200ECE6F200ECF6F200ED06F200ED16F42
:10AC6000200ED26FD36B200ED46F200ED56F200E26
:10AC7000D66F200ED76F200ED86F200ED96F200E02
:10AC8000DA6F200EDB6F4E0EDC6F6F0EDD6F200E65
:10AC9000DE6F200EDF6F200EE06F200EE16F200EC2
:10ACA000E26F200EE36F200EE46FE56B200EE66F7F
:10ACB000E76BE86BE96BEA6BEB6BEC6BED6BEE6BE8
:10ACC000EF6BF06BF16BF26BF36BF46BF56BF66B98
:10ACD000F76B200EF86FF96BFA6BFB6BFC6BFD6B7F
:10ACE000FE6BFF6B0301006B016B026B036B046B6C
:10ACF000056B066B076B086B096B200E0A6F0B6BFD
:10AD00000C6B0D6B0E6B0F6B106B116B126B136B6F
:10AD1000146B156B166B176B186B196B1A6B1B6B1F
:10AD2000200E1C6F1D6B1E6B1F6B206B216B226B2B
:10AD3000236B246B256B266B276B286B296B2A6B87
:10AD40002B6B2C6B2D6B200E2E6F2F6B306B316BA2
:10AD5000326B336B346B356B366B376B386B396BEF
:10AD60003A6B3B6B3C6B3D6B3E6B3F6B200E406F19
:10AD7000416B426B436B446B456B466B476B486B57
:10AD8000496B4A6B4B6B4C6B4D6B4E6B4F6B506B07
:10AD9000516B200E526F536B546B556B566B576B48
:10ADA000586B596B5A6B5B6B5C6B5D6B5E6B5F6B6F
:10ADB000606B616B626B636B200E646F656B666BBF
:10ADC000676B686B696B6A6B6B6B6C6B6D6B6E6BD7
:10ADD0006F6B706B716B726B736B746B756B200E3A
:10ADE000766F776B786B796B7A6B7B6B7C6B7D6B3B
:10ADF0007E6B7F6B806B816B826B836B846B856BEF
:10AE0000866B876B200E886F896B8A6B8B6B8C6B64
:10AE10008D6B8E6B8F6B906B916B926B936B946B56
:10AE2000956B966B976B986B996B200E9A6F9B6BDB
:10AE30009C6B9D6B9E6B9F6BA06BA16BA26BA36BBE
:10AE4000A46BA56BA66BA76BA86BA96BAA6BAB6B6E
:10AE5000200EAC6FAD6BAE6BAF6BB06BB16BB26B0A
:10AE6000B36BB46BB56BB66BB76BB86BB96BBA6BD6
:10AE7000BB6BBC6BBD6B200EBE6FBF6BC06BC16B81
:10AE8000C26BC36BC46BC56BC66BC76BC86BC96B3E
:10AE9000CA6BCB6BCC6BCD6BCE6BCF6B200ED06FF8
:10AEA000D16BD26BD36BD46BD56BD66BD76BD86BA6
:10AEB000D96BDA6BDB6BDC6BDD6BDE6BDF6BE06B56
:10AEC000E16B200EE26FE36BE46BE56BE66BE76B27
:10AED000E86BE96BEA6BEB6BEC6BED6BEE6BEF6BBE
:10AEE000F06BF16BF26BF36B200EF46FF56BF66B9E
:10AEF000F76BF86BF96BFA6BFB6BFC6BFD6BFE6B26
:10AF0000FF6B0401006B016B026B036B046B056B41
:10AF1000200E066F076B086B096B0A6B0B6B0C6BD3
:10AF20000D6B0E6B0F6B106B116B126B136B146B45
:10AF3000156B166B176B200E186F196B1A6B1B6B4A
:10AF40001C6B1D6B1E6B1F6B206B216B226B236BAD
:10AF5000246B256B266B276B286B296B200E2A6FC1
:10AF60002B6B426B436B010E446F010E456F020E5B
:10AF7000466F020E476F030E486F030E496F040EB3
:10AF80004A6F040E4B6F050E4C6F050E4D6F060E8B
:10AF90004E6F060E4F6F070E506F070E516F080E63
:10AFA000526F080E536F090E546F090E556F140E31
:10AFB000566F0A0E576F120E586F130E596F130EFD
:10AFC0005A6F0B0E5B6F0A0E5C6F120E5D6F0B0EED
:10AFD0005E6F0C0E5F6F0C0E606F0D0E616F0D0ECD
:10AFE000626F0E0E636F0E0E646F0F0E656F0F0EA5
:10AFF000666F100E676F100E686F110E696F110E7D
:10B000006A6F6B6B816B806B8D989698700ED36EA8
:10B01000400E9B6ED350F19E800ED56E9D8AA38A02
:10B02000C00EF212000196EF0FF06DEF10F0040E5B
:10B03000EA6E6C0EE96E06010F6B116B140E106F49
:10B04000000187EC0FF0A7EF11F0040EEA6E6C0E12
:10B05000E96EE26A310EE16EE752E6CFEEFFFCE107
:10B060000C0E04016C6F040EC86F6C0EC76F0001EC
:10B0700083EC12F0040EEA6E6C0EE96EE26A1F0EAB
:10B08000E16EE752E6CFEEFFFCE10A0E04016C6FC1
:10B09000040EC86F6C0EC76F000183EC12F01FEF37
:10B0A00013F07BEF13F0012C01D002D00AEF14F063
:10B0B000E5EC16F0020E0401826FFA0ECC6F00016F
:10B0C000B9EC0FF00401822FF8D7040E06010F6FC0
:10B0D0000001BCEC16F0060E06010F6F0001BCEC7F
:10B0E00016F082EF1EF0BAEF20F02BEF4CF01EB0FE
:10B0F00010D0895302E00AEF53F00101205303E01E
:10B1000000011DEF54F0010E0401CC6F0001B9ECF9
:10B110000FF00401802BD8B4812B8151000809E283
:10B12000FF0A03E180512C0804E2816B806B929846
:08B1300089780001D8D7030063
:020000040030CA
:0E00000000C81E1E0385B100FFC0FFE0FF40D8
:00000001FF
